:020000040800F2
:1000000000070020F5040008A92E0008612E000852
:10001000892E0008612E0008812E0008F7040008D0
:10002000F7040008F7040008F70400089D3E0008E4
:10003000F7040008F7040008F7040008F7040008B4
:10004000F7040008F7040008F7040008F7040008A4
:10005000F7040008F70400086D64000895640008C0
:10006000BD640008E56400080D650008F704000899
:10007000F7040008F7040008F7040008F704000874
:10008000F7040008F7040008F7040008152E00081C
:10009000412E0008512E0008F704000835650008BD
:1000A000F7040008F7040008F7040008F704000844
:1000B00009660008F7040008F7040008F7040008C0
:1000C000F7040008F7040008F7040008F704000824
:1000D000F7040008F7040008F7040008F704000814
:1000E00099650008F7040008F7040008F704000801
:1000F000F7040008F7040008F7040008F7040008F4
:10010000F7040008F7040008F7040008F7040008E3
:10011000F7040008F7040008F7040008F7040008D3
:10012000F7040008F7040008F7040008F7040008C3
:10013000F7040008F7040008F7040008F7040008B3
:10014000F7040008F7040008F7040008615A0008E3
:10015000F7040008F7040008F7040008F704000893
:10016000F7040008F7040008F7040008F704000883
:10017000F7040008F7040008F7040008F704000873
:10018000F7040008F7040008F7040008F704000863
:10019000F7040008F7040008F7040008F704000853
:1001A000F7040008F7040008F7040008F704000843
:1001B000F7040008F7040008F7040008F704000833
:1001C000F7040008F7040008F7040008F704000823
:1001D000F7040008F7040008F7040008F704000813
:1001E0005D18000800000000000000000000000092
:1001F00053B94AB9002908BF00281CBF4FF0FF318E
:100200004FF0FF3000F074B9ADF1080C6DE904CE89
:1002100000F006F8DDF804E0DDE9022304B07047E1
:100220002DE9F047089D04468E46002B4DD18A42A9
:10023000944669D9B2FA82F252B101FA02F3C2F1DC
:10024000200120FA01F10CFA02FC41EA030E94406D
:100250004FEA1C48210CBEFBF8F61FFA8CF708FB8E
:1002600016E341EA034306FB07F199420AD91CEB66
:10027000030306F1FF3080F01F81994240F21C8198
:10028000023E63445B1AA4B2B3FBF8F008FB1033E0
:1002900044EA034400FB07F7A7420AD91CEB040415
:1002A00000F1FF3380F00A81A74240F207816444E5
:1002B000023840EA0640E41B00261DB1D44000236A
:1002C000C5E900433146BDE8F0878B4209D9002DCE
:1002D00000F0EF800026C5E9000130463146BDE858
:1002E000F087B3FA83F6002E4AD18B4202D38242C2
:1002F00000F2F980841A61EB030301209E46002D71
:10030000E0D0C5E9004EDDE702B9FFDEB2FA82F2C5
:10031000002A40F09280A1EB0C014FEA1C471FFA23
:100320008CFE0126200CB1FBF7F307FB131140EA0A
:1003300001410EFB03F0884208D91CEB010103F1D7
:10034000FF3802D2884200F2CB804346091AA4B299
:10035000B1FBF7F007FB101144EA01440EFB00FE6D
:10036000A64508D91CEB040400F1FF3102D2A645D2
:1003700000F2BB800846A4EB0E0440EA03409CE771
:10038000C6F12007B34022FA07FC4CEA030C20FA1E
:1003900007F401FA06F31C43F9404FEA1C4900FA3E
:1003A00006F3B1FBF9F8200C1FFA8CFE09FB1811BB
:1003B00040EA014108FB0EF0884202FA06F20BD92E
:1003C0001CEB010108F1FF3A80F08880884240F27E
:1003D0008580A8F102086144091AA4B2B1FBF9F0C2
:1003E00009FB101144EA014100FB0EFE8E4508D9BD
:1003F0001CEB010100F1FF346CD28E456AD9023842
:10040000614440EA0840A0FB0294A1EB0E01A14226
:10041000C846A64656D353D05DB1B3EB080261EB94
:100420000E0101FA07F722FA06F3F1401F43C5E96E
:10043000007100263146BDE8F087C2F12003D840A4
:100440000CFA02FC21FA03F3914001434FEA1C47E6
:100450001FFA8CFEB3FBF7F007FB10360B0C43EAD8
:10046000064300FB0EF69E4204FA02F408D91CEB88
:10047000030300F1FF382FD29E422DD90238634486
:100480009B1B89B2B3FBF7F607FB163341EA034126
:1004900006FB0EF38B4208D91CEB010106F1FF3875
:1004A00016D28B4214D9023E6144C91A46EA00466C
:1004B00038E72E46284605E70646E3E61846F8E6FE
:1004C0004B45A9D2B9EB020864EB0C0E0138A3E747
:1004D0004646EAE7204694E74046D1E7D0467BE728
:1004E000023B614432E7304609E76444023842E7A0
:1004F000704700BF02E000F000F8FEE772B6374830
:1005000080F30888364880F3098836483649086001
:1005100040F20000CCF200004EF63471CEF2000141
:100520000860BFF34F8FBFF36F8F40F20000C0F23F
:10053000F0004EF68851CEF200010860BFF34F8FF5
:10054000BFF36F8F4FF00000E1EE100A4EF63C71E2
:10055000CEF200010860062080F31488BFF36F8F8D
:1005600004F046FF05F02AFE4FF055301F491B4AA4
:1005700091423CBF41F8040BFAE71D49184A9142E9
:100580003CBF41F8040BFAE71A491B4A1B4B9A423D
:100590003EBF51F8040B42F8040BF8E7002018495D
:1005A000184A91423CBF41F8040BFAE704F024FFDB
:1005B00005F058FE144C154DAC4203DA54F8041BF8
:1005C0008847F9E700F042F8114C124DAC4203DACB
:1005D00054F8041B8847F9E704F00CBF000700201B
:1005E000002300200000000808ED00E000010020CA
:1005F00000070020F86B000800230020B023002033
:10060000B023002048560020E0010008E401000863
:10061000E4010008E40100082DE9F04F2DED108AF7
:10062000C1F80CD0C3689D46BDEC108ABDE8F08FC0
:10063000002383F311882846A047002004F0E6F940
:10064000FEE704F03FF900DFFEE70000F8B501F037
:1006500017F904F067FE074604F0B6FE0546B8BB7E
:10066000204B9F4234D001339F4234D01E4B27F0A1
:10067000FF029A4232D1F8B200F00EFF2E4642F24B
:10068000107400F00FFF08B10024264601F0FAFCB8
:1006900020B1032000F07CF80024264635B1134B2E
:1006A0009F4203D004F088FE00242646002004F078
:1006B00043FE0EB100F082F801F094FA00F05EFF04
:1006C00001F044F9204600F0D5F800F077F8F9E79A
:1006D0002E460024D5E704460126D2E7064641F21D
:1006E0008834CEE7010007B0000008B0263A09B010
:1006F00008B501F0FDF8A0F120035842584108BDAB
:1007000007B541F21203022101A8ADF8043001F04F
:100710000DF903B05DF804FB38B5302383F311887D
:10072000174803680BB104F03DFA164A1448002339
:100730004FF47A7104F02CFA002383F31188124CE1
:10074000236813B12368013B2360636813B16368B6
:10075000013B63600D4D2B7833B963687BB9022090
:1007600001F0BAF9322363602B78032B07D1636859
:100770002BB9022001F0B0F94FF47A73636038BDF1
:10078000B023002019070008D0240020C82300202F
:10079000084B187003280CD8DFE800F008050208A1
:1007A000022001F08FB9022001F082B9024B002231
:1007B0005A607047C8230020D024002010B501F0F3
:1007C00061FC30B1244B03221A70244B00225A6082
:1007D00010BD234B234A1C4619680131F8D004335D
:1007E0009342F9D16268204B9A42F1D91F4B9B6822
:1007F00003F1006303F580339A42E9D204F0B0FDBF
:1008000004F0C2FD002001F0BBF80220FFF7C0FF9A
:10081000174B1A6C00221A64196E1A66196E596CFD
:100820005A64596E5A665A6E1A6942F000521A6139
:100830001A6922F000521A611B6972B64FF0E02368
:100840003021C3F8084DD4E9003281F311889D4668
:1008500083F308881047BBE7C8230020D02400207A
:100860000000010820000108FFFF0008002300200D
:10087000003802402DE9F04F93B0AC4B009020229D
:10088000FF210AA89D6801F057F9A94A1378A3B976
:10089000A848012103601170302383F31188036895
:1008A0000BB104F07FF9A44AA24800234FF47A71F7
:1008B00004F06EF9002383F31188009B13B19F4B62
:1008C000009A1A609E4A009C1378032B1EBF0023D7
:1008D00013709A4A4FF0000A18BF5360D346564629
:1008E000D146012001F0EEF824B1944B1B68002B97
:1008F00000F01582002000F0FBFF0390039B002B0B
:1009000001DA00F083FE039B002BEDDB012001F0F8
:10091000CFF8039B213B162BE3D801A252F823F01A
:100920007D090008A5090008390A0008E308000845
:10093000E3080008E3080008C30A0008930C000855
:10094000AD0B00080F0C0008370C00085D0C000808
:10095000E30800086F0C0008E3080008E10C000839
:100960001D0A0008E3080008250D00088909000891
:100970001D0A0008E30800080F0C00080220FFF71A
:10098000B7FE002840F0F581009B0221BAF1000F6C
:1009900008BF1C4605A841F21233ADF8143000F030
:1009A000C5FF9EE74FF47A7000F0A2FF071EEBDB55
:1009B0000220FFF79DFE0028E6D0013F052F00F240
:1009C000DA81DFE807F0030A0D10133605230593DB
:1009D000042105A800F0AAFF17E054480421F9E714
:1009E00058480421F6E758480421F3E74FF01C0863
:1009F000404600F0C7FF08F104080590042105A84F
:100A000000F094FFB8F12C0FF2D1012000FA07F7A3
:100A100047EA0B0B5FFA8BFB4FF0000901F0D8F8A7
:100A200026B10BF00B030B2B08BF0024FFF768FE69
:100A300057E746480421CDE7002EA5D00BF00B0365
:100A40000B2BA1D10220FFF753FE074600289BD0B5
:100A5000012000F095FF0220FFF79AFE00261FFA02
:100A600086F8404600F09CFF044690B100214046C5
:100A700000F0AEFF01360028F1D1BA46044641F23B
:100A80001213022105A8ADF814303E4600F04EFFC7
:100A900027E70120FFF77CFE2546244B9B68AB42ED
:100AA00007D9284600F06EFF013040F06781043519
:100AB000F3E7234B00251D70204BBA465D603E4690
:100AC000ACE7002E3FF460AF0BF00B030B2B7FF471
:100AD0005BAF0220FFF75CFE322000F009FFB0F1AF
:100AE0000008FFF651AF18F003077FF44DAF0F4A2F
:100AF000926808EB050393423FF646AFB8F5807F56
:100B00003FF742AF124B0193B84523DD4FF47A70A3
:100B100000F0EEFE0390039A002AFFF635AF019B2A
:100B2000039A03F8012B0137EDE700BF00230020F3
:100B3000CC240020B023002019070008D024002076
:100B4000C823002004230020082300200C230020B9
:100B5000CC230020C820FFF7CBFD074600283FF438
:100B600013AF1F2D11D8C5F1200242450AAB25F065
:100B7000030028BF424683490192184400F0B6FFA3
:100B8000019A8048FF2100F0D7FF4FEAA8037D4972
:100B90000193C8F38702284600F0D6FF06460028D6
:100BA0003FF46DAF019B05EB830537E70220FFF7AC
:100BB0009FFD00283FF4E8AE00F02AFF00283FF434
:100BC000E3AE0027B846704B9B68BB4218D91F2F75
:100BD00011D80A9B01330ED027F0030312AA134445
:100BE00053F8203C05934046042205A901F002FA7F
:100BF00004378046E7E7384600F0C4FE0590F2E788
:100C0000CDF81480042105A800F090FE06E700232B
:100C1000642104A8049300F07FFE00287FF4B4AEA2
:100C20000220FFF765FD00283FF4AEAE049800F007
:100C3000D7FE0590E6E70023642104A8049300F0A2
:100C40006BFE00287FF4A0AE0220FFF751FD0028C4
:100C50003FF49AAE049800F0D3FEEAE70220FFF7D3
:100C600047FD00283FF490AE00F0E2FEE1E70220ED
:100C7000FFF73EFD00283FF487AE05A9142000F0E1
:100C8000DDFE04210746049004A800F04FFE39461B
:100C9000B9E7322000F02CFE071EFFF675AEBB0749
:100CA0007FF472AE384A926807EB090393423FF62D
:100CB0006BAE0220FFF71CFD00283FF465AE27F065
:100CC00003074F44B9453FF4A9AE484600F05AFE29
:100CD0000421059005A800F029FE09F10409F1E7B7
:100CE0004FF47A70FFF704FD00283FF44DAE00F09A
:100CF0008FFE002844D00A9B01330BD008220AA99A
:100D0000002000F021FF00283AD02022FF210AA86D
:100D100000F012FFFFF7F4FC1C4803F07DFE13B057
:100D2000BDE8F08F002E3FF42FAE0BF00B030B2B22
:100D30007FF42AAE0023642105A8059300F0ECFDA2
:100D4000074600287FF420AE0220FFF7D1FC804642
:100D500000283FF419AEFFF7D3FC41F2883003F0CE
:100D60005BFE059800F066FF464600F031FF3C460A
:100D7000B7E5064652E64FF0000905E6BA467EE6BC
:100D800037467CE6CC23002000230020A08601000B
:100D9000094A136849F2690099B21B0C00FB013340
:100DA0001360064B186844F2506182B2000C01FBDC
:100DB0000200186080B2704718230020142300201E
:100DC00010B500211022044600F0B6FE034B03CB01
:100DD000206061601868A06010BD00BF107AFF1F1E
:100DE0002DE9F041ADF5507D0DF13C086EAC40F2BF
:100DF000751207460D4610A80021C8F8001000F033
:100E00009BFE4FF4C4720021204600F095FE02F0D4
:100E100053F8254B4FF47A72B0FBF2F0186093E868
:100E20000700022384E807000DF5ED702382FFF729
:100E3000C7FF4FF203631D49238406A805F0F4FCA5
:100E4000202384F832310DF2EB2606AB0DF1380C7D
:100E50001A4603CA624530607160134606F10806FF
:100E6000F6D141460122204600F0E6FE002303931E
:100E7000AB7E029305F11903019380B20123CDE902
:100E800004800093E97E06A3D3E90023384602F0EC
:100E9000DBFB0DF5507DBDE8F08100BFAFF30080B6
:100EA0009E6AC421818A46EED82400203868000852
:100EB0002DE9F0412C4C237ADAB080460D465BBB1D
:100EC00027A9284600F0C8FF0746002842D19DF810
:100ED0009D60C82E3ED801464FF4A662204600F021
:100EE0002BFE4FF48073C4F8F8314FF40073C4F84C
:100EF0000C334FF44073C4F8203432460DF19E0198
:100F000004F1090000F0F2FD26449DF89C30777250
:100F100023720BB9EB7E23728122002106AC27A835
:100F200000F00AFE0122214627A800F0D1FF00238D
:100F30000393AB7E029305F1190380B2019328233A
:100F4000CDE904400093E97E05A3D3E900234046A0
:100F500002F07AFB5AB0BDE8F08100BFAFF3008029
:100F600026417272DF25D7B7F0450020F0B5254E37
:100F70004FF48A7505FB0065F1B096F8D83085F816
:100F8000DC300024D822214685F8E8403AA800F059
:100F9000D3FD06F1090000F0C7FDD5F8E4308DF867
:100FA000F000C2B206AF06F109010DF1F100CDE982
:100FB0003A3400F09BFD394601223AA800F0B4FF14
:100FC00080B2CDE9047008230127CDE9023706F18C
:100FD000D803019330230093317A0B4807A3D3E958
:100FE000002302F031FBA04206DD01F065FFC5F8E9
:100FF000E000384671B0F0BD2046FBE778F6339F3D
:1010000093CACD8DF0450020F03400202DE9F04149
:101010001D4D1E4E1E4F86B0284602F041FB034672
:1010200058B30024CDE90344ADF81440027B8DF899
:10103000142099684068029403AA03C21B68DFF871
:10104000548043F00043029301F038FF821941F1CC
:101050000003009402A9384601F0FAF9A04205DD28
:10106000284602F021FB88F80040D5E798F80030C8
:10107000072B05D8013388F8003006B0BDE8F081B1
:10108000014802F011FBF8E7F034002040420F0065
:1010900020350020254B002070B50D4614461E4615
:1010A00002F02EFA50B9022E10D1012C0ED112A34B
:1010B000D3E90023C5E90023012007E0282C10D044
:1010C00005D8012C09D0052C0FD0002070BD302C84
:1010D000FBD10BA3D3E90023ECE70BA3D3E9002357
:1010E000E8E70BA3D3E90023E4E70BA3D3E900234C
:1010F000E0E700BFAFF30080401DA12026812A0B4E
:1011000078F6339F93CACD8D9E6AC421818A46EEBC
:1011100026417272DF25D7B7F017304A39059E563F
:1011200038B505460E4C0021013500F051FCA4F8FD
:101130002C55B4F82C0500F033FC78B1B4F82C052C
:1011400000F03EFC014648B9B4F82C0500F040FC24
:10115000B4F82C350133A4F82C35EAE738BD00BFCC
:10116000F045002010B50A4B0A4A1A6003F5805377
:1011700093F860203AB9DC6D2CB1204601F000F8FC
:10118000204605F091FABDE81040034800F0F8BF92
:1011900020350020F8680008684500202DE9F04F50
:1011A0008FB000AF05460C4602F0AAF9002849D1DD
:1011B000237E022B1BD1E38A012B18D101F07CFE88
:1011C0000646FFF7E5FD03464FF4C870DFF8C4821A
:1011D000B3FBF0F206F5167602FB103316FA83F332
:1011E000C8F80030E37E33B9A34B00221A703C37B5
:1011F000BD46BDE8F08F07F12401204600F0EAFD6E
:101200000028F4D107F11400FFF7DAFD97F8264023
:1012100007F11401224607F1270005F08FFA002894
:10122000E2D10F2C08D8944B1C70D8F80030A3F5ED
:101230001673C8F80030DAE797F82410284602F051
:1012400057F9D4E7E38A282B2BD010D8012B23D0D1
:10125000052BCCD1BFF34F8F8849894BCA6802F464
:10126000E0621343CB60BFF34F8F00BFFDE7302B2D
:10127000BDD1844EE17E327A9142B8D1607E314652
:10128000002291F8DC50854200F0A5800132042A4A
:1012900001F58A71F5D1AAE721462846FFF7A0FD9E
:1012A000A5E721462846FFF703FEA0E7B2F8EC5079
:1012B0007B6005F103094FEA99094FEA8902D11DC4
:1012C000C908A8EBC1039D46EB460021584600F033
:1012D00033FC04F1EE012A463144584600F006FC86
:1012E0007B6813B9012000F04BFB96F8D20000F0A8
:1012F00057FB044630B9307200F08AFB204600F0FC
:101300003FFBB1E0D6F8D4203AB996F8D200B6F84F
:101310002C25824201D8FFF703FFD6F8D4202A44B7
:10132000944208D296F8D200B6F82C2501308242B9
:1013300001D8FFF7F5FE70685FFA89F2594600F0B0
:1013400003FC08B9C54679E0726896F8D2002A44D1
:101350007260D6F8D42005EB0209C6F8D49000F0EC
:101360001FFB814509D396F8D220D6F8D40001326C
:10137000001B86F8D220C6F8D400FF2D0FD8002419
:10138000347200F045FB204600F0FAFA00F07AFED5
:101390003D4B188108B9FFF711FAC54627E7BB682E
:1013A00096F8D9000AFB0362FB68D2F8E41082F8D1
:1013B000E83001F58061C2F8E030C2F8E410FFF7D0
:1013C000D5FDFFF723FE96F8D920013202F0030283
:1013D00086F8D920B6E74FF48A7A0AFB02F505F1C0
:1013E000EA013144204600F0CBFDF86000287FF48C
:1013F000FEAE3544012285F8E82001F05DFDD5F808
:10140000E020D6ED007ADFED216A801A192838BF76
:10141000192040F6B832904228BF1046B8EE677ADD
:1014200007EE900AF8EEE77A67EEA67ADFED186A23
:10143000E7EE267AFCEEE77AC6ED007A96F8D93028
:10144000BB60BA6873680AFB02F4321992F8E810BC
:1014500059B1D2F8E4108B42E8463FF427AF00219F
:1014600082F8E810C2F8E010C5467368064A9B0A85
:1014700001331381BBE600BFE934002000ED00E03A
:101480000400FA05F0450020D8240020CDCCCC3D46
:101490006666663FEC340020014B1870704700BF51
:1014A000E424002030B54FF000542B4B22689A42C0
:1014B00085B007D003F092FF044620BB00242046ED
:1014C00005B030BD254B627D25481A70237D03721F
:1014D0004FF48073C0F8F8314FF40073C0F80C3348
:1014E00000254FF44073C0F820341E49C0F8E45082
:1014F000C922093000F0FAFA2046E022294600F01D
:101500001BFB0124DBE7184A184D136C43F00073F2
:101510001364AA6D164B9A42D0D12B6E013B7E2BE1
:10152000CCD8144A07CA01AB83E807001846032148
:1015300000F076FD6B6D83424FF00003BED12A6D43
:101540008A4201BFAB65054B2A6E1A7003BF0A4B76
:10155000EA6D1A601C46B2E79AAD44C5E424002047
:10156000F0450020160000200038024000660040D0
:101570005041A0B0586600401023002037B51A4DE6
:1015800000F080FD02236B71184B28811968184800
:10159000012201F02FFB00230193164B1649009303
:1015A0001648174B4FF4805201F07AFF154B19780B
:1015B00011B1124801F09CFF01F07EFC0446FFF7D8
:1015C000E7FB4FF4C873B0FBF3F202FB130304F51F
:1015D000167010FA83F00C4B186003F0F5FE08B19A
:1015E0000F232B8103B030BDD8240020102300200E
:1015F0002035002099100008E8240020F034002055
:101600009D110008E4240020EC3400202DE9F04F67
:101610002DED028B0FF23829D9E90089834C93B064
:101620000BAE9FED7E8BFFF7F1FC814FDFF828A218
:1016300000230A93ADF834300B9373604FF0000B26
:101640005B468DED008B01250DF11D0207A9384683
:101650008DF81C508DF81DB001F07CFA9DF81C30FF
:10166000002B40F0A580204601F04AFF06460028E6
:1016700045D1704F01F020FC3B6898423FD301F008
:101680001BFC8246FFF784FB4FF4C873B0FBF3F2F8
:1016900002FB13030AF5167010FA83F03860664FE8
:1016A00097F800B0CBF1100ABBF1000F14BF33461E
:1016B0002B465FFA8AFA0EA88DF82830FFF780FBD8
:1016C000BAF1060F28BF4FF0060A0EAB03EB0B0171
:1016D00052460DF1290000F009FA0AAB03931823D2
:1016E00002930AF10102554BD2B2CDE900530492A4
:1016F00020464CA3D3E9002301F048FF3E7001F0DF
:10170000DBFB4F4A4F4D1368C31AB3F57A7F2ED3D4
:10171000106001F0D3FB02460B46204601F0CEFFDD
:10172000204601F0EDFE10B32B7A474E002B14BF7C
:1017300003230223737101F0BFFB0EAF4FF47A73E2
:101740000122B0FBF3F039463060304600F01AFB5E
:10175000182302933D4B019380B240F25513CDE91B
:101760000370009342464B46204601F00FFF2B7A50
:1017700093B101F0A1FB002607464FF48A7A95F851
:10178000D900304400F003000AFB005393F8E8202E
:1017900092B30136042EF2D1C82003F03DF92B7A22
:1017A000002B7FF43DAF13B0BDEC028BBDE8F08F92
:1017B000DAF8143083F48043CAF814305946102202
:1017C0000EA800F0B9F90DF11E0308AA0AA93846BF
:1017D00000F03CFF96E803000FAB83E803009DF8A0
:1017E00034308DF844300A9B0E930EA9DDE90823AE
:1017F000204602F037F921E7D3F8E02042B12B6808
:10180000FA2B38BFFA23BA1A0533B2EB430FC0D311
:10181000FFF7ACFB0028BCD1BEE700BF0000000012
:1018200000000000401DA12026812A0BF03400207A
:1018300020350020EC340020E9340020E83400207A
:10184000204B0020F0450020D8240020244B00200D
:10185000F1C6A7C1D068080F0000024008B50548CE
:1018600000F08EFFBDE80840034A0449002004F060
:1018700015BF00BF20350020604B00206511000817
:101880007047000070B50F4B1B780133DBB2012BA2
:101890000C4611D80C4D29684FF47A730E6AA2FBDE
:1018A0000332014622462846B047844204D1074B02
:1018B00000221A70012070BD4FF4FA7003F0ACF8EA
:1018C0000020F8E71C230020D84D0020544B0020B6
:1018D00070B504464FF47A76412C254628BF412541
:1018E00006FB05F003F098F8641BF5D170BD00000D
:1018F00007B50023024601210DF107008DF80730DE
:10190000FFF7C0FF20B19DF8070003B05DF804FBAE
:101910004FF0FF30F9E700000A4608B50421FFF751
:10192000B1FF80F00100C0B2404208BD30B4054CA8
:101930002368DD69044B0A46AC460146204630BCAC
:10194000604700BFD84D0020A086010070B503F0AD
:1019500083FB094E094D3080002428683388834278
:1019600008D903F073FB2B6804440133B4F5803FBE
:101970002B60F2D370BD00BF564B0020284B0020D7
:1019800003F018BC00F1006000F58030006870477B
:1019900000F10060920000F5803003F0A3BB00006E
:1019A000054B1A68054B1B889B1A834202D91044C9
:1019B00003F04CBB00207047284B0020564B002002
:1019C000024B1B68184403F049BB00BF284B0020A2
:1019D000024B1B68184403F059BB00BF284B002082
:1019E00010F003030AD1B0F5047F05D200F10050D6
:1019F000A0F51040D0F80038184670470023FBE7E8
:101A000000F10050A0F51040D0F8100A7047000017
:101A1000064991F8243033B10023086A81F8243054
:101A20000822FFF7B5BF0120704700BF2C4B0020F4
:101A3000014B1868704700BF002004E070B5194BD7
:101A40001D68194B0138C5F30B0408442D0C042202
:101A50001E88A6420BD15C680A46013C82421346AE
:101A60000FD214F9016F4EB102F8016BF6E7013A9B
:101A700003F10803ECD181420B4602D22C2203F879
:101A8000012B0A4A05241688AE4204D1984284BF2D
:101A9000967803F8016B013C02F10402F3D1581A65
:101AA00070BD00BF002004E09C6800088868000842
:101AB000022802BF024B4FF080429A61704700BF7C
:101AC00000000240022802BF024B4FF480429A619C
:101AD000704700BF00000240022801BF024A53695C
:101AE00083F48043536170470000024010B5002327
:101AF000934203D0CC5CC4540133F9E710BD00001D
:101B000010B5013810F9013F3BB191F900409C42FA
:101B100003D11AB10131013AF4E71AB191F9002069
:101B2000981A10BD1046FCE703460246D01A12F977
:101B3000011B0029FAD1704702440346934202D0A8
:101B400003F8011BFAE770472DE9F8431F4D1446CF
:101B500095F824200746884652BBDFF870909CB366
:101B600095F824302BB92022FF2148462F62FFF739
:101B7000E3FF95F82400C0F10802A24228BF2246E4
:101B8000D6B24146920005EB8000FFF7AFFF95F813
:101B90002430A41B1E44F6B2082E17449044E4B22D
:101BA00085F82460DBD1FFF733FF0028D7D108E0A8
:101BB0002B6A03EB82038342CFD0FFF729FF002873
:101BC000CBD10020BDE8F8830120FBE72C4B00209F
:101BD000024B1A78024B1A70704700BF544B00201A
:101BE0001C23002010B5104C104802F045FA214685
:101BF0000E4802F06DFA2468626DD2F8043843F0A2
:101C00000203C2F804384FF47A70FFF761FE084906
:101C1000204602F063FB626DD2F8043823F0020321
:101C2000C2F8043810BD00BFE4690008D84D002098
:101C3000EC690008704700002DE9F0470D460446A6
:101C400000219046284640F27912FFF775FF23469F
:101C500020220021284601F0A7FE231D0222202178
:101C6000284601F0A1FE631D03222221284601F02F
:101C70009BFEA31D03222521284601F095FE04F1B9
:101C8000080310222821284601F08EFE04F11003DB
:101C900008223821284601F087FE04F111030822AA
:101CA0004021284601F080FE04F112030822482159
:101CB000284601F079FE04F1140320225021284621
:101CC00001F072FE04F1180340227021284601F051
:101CD0006BFE04F120030822B021284601F064FEC7
:101CE00004F121030822B821284601F05DFE04F129
:101CF0002207C0263B46314608222846083601F016
:101D000053FEB6F5A07F07F10107F3D104F13203CA
:101D100008223146284601F047FE002704F1330A25
:101D200094F832304FEAC7099F4209F5A47615D3DB
:101D3000B8F1000F08D1314604F5997307222846FF
:101D400001F032FE09F24F16274694F832213B1B70
:101D500093420CD3F01DC008BDE8F0870AEB0703DF
:101D600008223146284601F01FFE0137D8E707F266
:101D7000331331460822284601F016FE0836013793
:101D8000E3E7000013B5044608460021016023463E
:101D9000C0F803102022019001F006FE0198231DD7
:101DA0000222202101F000FE0198631D032222215E
:101DB00001F0FAFD0198A31D0322252101F0F4FD95
:101DC000019804F108031022282101F0EDFD0720FD
:101DD00002B010BDF7B50023047F00910E46072224
:101DE0001946054601F0A4FC731C00930122002350
:101DF0000721284601F09CFCC4B9B31C00930522BE
:101E000023460821284601F093FC0D243746B2787A
:101E1000BB1B934211D32B7FA88A0734E408BBB9BC
:101E2000844294BF0020012003B0F0BDAB8ADB00E8
:101E3000083BDB08B3700824E8E7FB1C009321464D
:101E400000230822284601F073FC08340137DEE73E
:101E5000201A18BF0120E7E7F7B50023047F00919F
:101E60000E4608221946054601F062FC731CC4B9EF
:101E70000822009311462346284601F059FC1024FD
:101E8000012372785F1C013B934211D32B7FA88AF8
:101E90000734E408BBB9844294BF0020012003B09A
:101EA000F0BDAB8ADB00083BDB0873700824E7E772
:101EB000F3190093214600230822284601F038FC3C
:101EC00008343B46DDE7201A18BF0120E7E7000091
:101ED000F8B50E4605461446002181223046FFF72C
:101EE0002BFE2B4608220021304601F05DFD7CB917
:101EF0006B1C07220821304601F056FD0F240123F8
:101F00006A785F1C013B934204D3E01DC008F8BD12
:101F10000824F4E7EB1921460822304601F044FD7D
:101F200008343B46ECE70000F8B50E46054614467B
:101F30000021CE223046FFF7FFFD2B46282200214C
:101F4000304601F031FD7CB905F108030822282153
:101F5000304601F029FD30242F462A7A7B1B93421C
:101F600004D3E01DC008F8BD2824F5E707F10903F4
:101F700021460822304601F017FD08340137ECE70E
:101F8000F7B5047F00910E4601231022002105467B
:101F900001F0CEFBC4B9B31C0093092223461021E3
:101FA000284601F0C5FB192437467288BB1B9A42AC
:101FB00011D82B7FA88A0734E408BBB9844294BFA8
:101FC0000020012003B0F0BDAB8ADB00103BDB0832
:101FD00073801024E8E73B1D00932146002308226C
:101FE000284601F0A5FB08340137DEE7201A18BFA8
:101FF0000120E7E730B5094D0A4491420DD011F8B0
:10200000013B5840082340F30004013B2C4013F0EF
:10201000FF0384EA5000F6D1EFE730BD2083B8ED2E
:10202000F7B54FF0FF33DFF854C0DFF854E000EBB2
:1020300081011A4688421CD050F8044B019401AF2C
:10204000042417F8015B82EA05620825DB181646AE
:1020500005F1FF355241002EBCBF83EA0C0382EA32
:102060000E0215F0FF05F1D1013C14F0FF04E8D198
:10207000E0E7D843D14303B0F0BD00BF9336EAA9EF
:10208000EBE1F042F7B5384A106851686B4603C37C
:102090006A4636493648082304F060FB04460028A7
:1020A00033D10A25334A106851686B4603C36A4628
:1020B00031492F48082304F051FB0446002849D039
:1020C0000369B3F5702F45D8B0F8661040F2F632C8
:1020D00091423FD1294A024402F15C018B4239D33B
:1020E0005C3B234900209E1AFFF784FF32460746D7
:1020F00004F164010020FFF77DFFA3689F4229D10E
:10210000E368984208BF002524E00369B3F5702F07
:1021100027D8418B40F2F632914220D1174A02442F
:1021200002F110018B4218D3103B114900209D1A77
:10213000FFF760FF2A46064604F118010020FFF76A
:1021400059FFA3689E4202D1E368984201D00D2551
:10215000A8E70025284603B0F0BD1025A2E70C250E
:10216000A0E70B259EE700BFBC680008DCFF0E005F
:1021700000000108C568000890FF0E000800FFF786
:1021800010B5037C044613B9006804F0CFFA20466A
:1021900010BD00000023BFF35B8FC360BFF35B8FF4
:1021A000BFF35B8F8360BFF35B8F7047BFF35B8FC1
:1021B0000068BFF35B8F704770B505460C30FFF7C2
:1021C000F5FF05F1080604463046FFF7EFFFA04291
:1021D00006D930466D68FFF7E9FF2544281A70BD1F
:1021E0003046FFF7E3FF201AF9E7000070B5054617
:1021F000406898B105F10800FFF7D8FF05F10C061B
:1022000004463046FFF7D2FF8442304694BF6D68E3
:102210000025FFF7CBFF013C2C44201A70BD0000C5
:1022200038B50C460546FFF7C7FFA04210D305F1AD
:102230000800FFF7BBFF04446868B4FBF0F100FB43
:102240001144BFF35B8F0120AC60BFF35B8F38BDDF
:102250000020FCE72DE9F041144607460D46FFF744
:10226000C5FF844228BF0446D4B1B84658F80C6B69
:102270004046FFF79BFF3044286040467E68FFF7EA
:1022800095FF331A9C4203D86C600120BDE8F081B1
:102290006B60A41B3B68AB602044E8600220F5E75C
:1022A0002046F3E738B50C460546FFF79FFFA042EE
:1022B00010D305F10C00FFF779FF04446868B4FB04
:1022C000F0F100FB1144BFF35B8F0120EC60BFF322
:1022D0005B8F38BD0020FCE72DE9FF418846694649
:1022E0000746FFF7B7FF6C4606B204EBC6060025AB
:1022F000B44209D06268206808EB0501FFF7F6FBDD
:10230000636808341D44F3E729463846FFF7CAFFDF
:10231000284604B0BDE8F081F8B505460C300F46FC
:10232000FFF744FF05F1080604463046FFF73EFF7D
:10233000A042304688BF6C68FFF738FF201A38602B
:1023400020B130462C68FFF731FF2044F8BD000073
:1023500073B5144606460D46FFF72EFF844228BF8C
:1023600004460190DCB101A93046FFF7D5FF019B7F
:1023700033B93268C5E90233C5E9002401200CE015
:102380009C4238BF01942860019868608442F5D966
:102390003368AB60241AEC60022002B070BD2046A6
:1023A000FBE700002DE9FF410F466946FFF7D0FF2C
:1023B0006C4600B204EBC0050026AC4209D0D4F84C
:1023C000048054F8081BB8194246FFF78FFB4644B7
:1023D000F3E7304604B0BDE8F081000038B50546AB
:1023E000FFF7E0FF044601462846FFF719FF2046A5
:1023F00038BD0000302383F3118862B670470000B7
:10240000002383F3118862B67047000010B402689D
:1024100054681A4623465DF8044B1847012070475C
:102420000020704700207047704700000020704770
:102430000E20704700F5805090F8C800C0F34000AF
:102440007047000000F5805090F9C9007047000007
:10245000F7B50C68BDF8207014F000541E466FD11B
:102460000B7B082B6CD8FFF7C5FF4569AB685B0198
:102470000CD4AB681B0108D4AC6814F080545DD157
:10248000FFF7BEFF204603B0F0BD01240B6804F146
:10249000180C002BB8BFDB004FEA0C1CB4BF43F094
:1024A00004035B0545F80C300B680FFA84FC13F04D
:1024B000804F18BF05EB0C1E05EB0C1C1EBFDEF891
:1024C000803143F00203CEF880310B7BCCF88431AD
:1024D00005EB04158B68C5F88C314B68C5F888315D
:1024E000DCF8803143F00103CCF8803100EB441577
:1024F00041F268031D4403EB44130344C5E900267D
:1025000008330D4601F10C0C55F804EB43F804EBCD
:102510006545F9D184342D881D8000EB441407F003
:102520000303257925F00B052B432371FFF768FF83
:102530000097334600F0E2FC0120A4E70224A5E75F
:102540004FF0FF309FE7000013B500F58054019174
:10255000E06DFFF74BFE1F280AD90199E06D20229C
:10256000FFF7BAFEA0F120035842584102B010BD57
:102570000020FBE708B500F58050FFF73BFFC06D7A
:10258000FFF708FEBDE80840FFF73ABF00220260EF
:10259000828142608260704710B500220023C0E94A
:1025A00000230023044603810C30FFF7EFFF204691
:1025B00010BD0000F0B5054600F580500C4690F8BF
:1025C000C83013F0040FC3F3800108BF114661F354
:1025D000820304F1840680F8C83005EB461389B005
:1025E0001B79D8072ED57AB319072DD46846FFF783
:1025F000D3FF05EB441303F5835303F1180703AA34
:10260000103318685968144603C40833BB42224685
:10261000F7D1186820609B88A380DDE90E23CDE9FF
:1026200000230123ADF808302B686946DB6B284690
:10263000984705EB46152B791A075CBF43F0080352
:102640002B7101E0002AF4D109B0F0BD2DE9F0476B
:10265000074688B007F5805468469A468846FFF7D3
:10266000C9FE9146FFF798FFE06DFFF7A5FD1F2813
:1026700029D9E06D20226946FFF7B0FE202822D13B
:1026800003AD444605AB2E4603CE9E4220606160FA
:10269000354604F10804F6D130682060B388A38081
:1026A000DDE90023C9E90023BDF80830AAF80030AD
:1026B000FFF7A6FE4A4653464146384608B0BDE8F5
:1026C000F04700F009BCFFF79BFE002008B0BDE812
:1026D000F08700002DE9F84F0023C0E90133254BB6
:1026E000044640F8183B0F46FFF750FF04F128005E
:1026F000FFF752FF04F1480804F5825546460835B5
:1027000030462036FFF748FFAE42F9D104F5805538
:102710004FF480534FF00009C5E91339C5F84880DC
:102720000123EE6504F5875804F58456C5F85490E6
:1027300085F8583085F86030083608F108084FF001
:10274000000A4FF0000B46E908ABA6F11800FFF7AE
:102750001DFF203646F8289C4645F4D185F8C970FF
:1027600017B1054800F0A2FB044B63612046BDE8A9
:10277000F88F00BFF8680008D068000800640040C7
:1027800010B5044B197804464A1C1A70FFF7A2FFD3
:10279000204610BD5C4B00202DE9F047002950D0A9
:1027A000294B2A4FB7FBF1F599428CBF0A2311231D
:1027B000581EB5FBF3FC03FB1C53C4B22BB102281B
:1027C0000346F5D80020BDE8F0870CF1FF36B6F5DA
:1027D000806FF7D2C4EBC40E0EF103034FEAE30996
:1027E000C3F3C703A4EB030809F1010A4FF47A7598
:1027F0005FFA88F009FB05555AFA88F8B5FBF8F539
:10280000B5F5617FC1BF0EF1FF33C3F3C703E01A13
:10281000C0B25C1C50FA84F40CFB04F4B7FBF4F473
:10282000A142CFD1013BDBB20F2BCBD80138C0B2D4
:102830000728C7D80021107116809170D37001202D
:10284000C1E70846BFE700BF3F420F0080DE8002BD
:1028500070B505460E464FF47A746B695B6803F0F9
:102860000103B34207D04FF47A7002F0D5F8013C6F
:10287000F3D1204670BD0120FCE7000030B542696D
:10288000936913F0700F16D000230B4C936103F182
:10289000840200EB421211794D0709D5890707D54B
:1028A000416954F823508D60117941F00401117190
:1028B0000133032BEBD130BDE468000873B51D462E
:1028C000436916469A68D207044609D59A680121D9
:1028D0009960C2F34002CDE900650021FFF76AFE6E
:1028E00063699A68D1050BD59A684FF48071996035
:1028F000C2F34022CDE9006501212046FFF75AFED0
:1029000063699A68D2030BD59A684FF48031996055
:10291000C2F34042CDE9006502212046FFF74AFE9E
:10292000204602B0BDE87040FFF7A8BFF8B50446E6
:10293000466900296CD106F10C07386880076AD017
:1029400006EB01153868D5F8B00110F0040FD5F882
:10295000B0011ABFC00840F00040400DA061D5F89A
:10296000B0C11CF0020F1CBF40F08040A061D5F840
:10297000B40106EB011100F00F0084F82400D1F837
:10298000B8012077D1F8B801000A6077D1F8B80112
:10299000000CA077D1F8B801000EE077D1F8BC01A7
:1029A00084F82000D1F8BC01000A84F82100D1F895
:1029B000BC01000C84F82200D1F8BC11090E84F887
:1029C00023103821396004F1340004F1180104F1B6
:1029D000240551F8046B40F8046BA942F9D1098829
:1029E0000180C4E90A2321460023238651F8283BAD
:1029F0002046DB6B984704F58052204692F8C83099
:102A000043F0040382F8C830BDE8F840FFF736BF52
:102A100006F1100791E7F8BD10B5044600F04EFA34
:102A200002460B4652EA030102D0013A63F1000369
:102A30000449086820B12146BDE81040FFF776BF81
:102A400010BD00BF584B0020F8B500F583511E465D
:102A5000FFF7D0FCDFF844C00831002404F18405FE
:102A600000EB45152B795F070ED4DB060CD5D1E9B9
:102A700000739742B34107D243695CF824709F60AA
:102A80002B7943F004032B710134032C01F1200155
:102A9000E4D1BDE8F840FFF7B3BC00BFE46800082C
:102AA00008B5FFF7A7FCFFF7E9FEBDE80840FFF710
:102AB000A7BC0000F8B543690546986800F0E050EF
:102AC000B0F1E05F0F461FD0E8B1FFF793FC05F5CA
:102AD00083541034002606F1840305EB43131B795D
:102AE0001A0706D50136032E04F12004F3D1012084
:102AF00007E05B07F6D42146384600F039FA002893
:102B0000F0D1FFF77DFCF8BD0120FCE700F5805017
:102B100008B5FFF76FFCC06DFFF74EFBFFF770FCC9
:102B200043090CBF0120002008BD0000F8B51D4678
:102B3000002313700F4606461446FFF7E7FF80F0A8
:102B40000100387025B129463046FFF7B3FF2070E9
:102B5000F8BD00002DE9B8410C4615461F468046D9
:102B600000F0ACF90B462178024609B9287850B13B
:102B70004046FFF769FFFFF793FF3B462A46214691
:102B8000FFF7D4FF0120BDE8B881000010B5FFF7C2
:102B900031FC174B1A6C42F000721A641A6A42F048
:102BA00000721A621A6A00F5805422F000721A62EA
:102BB000FFF726FC94F8C830DB0718D4B9B103211D
:102BC0001320FFF717FC01F0C7F90321142001F0CF
:102BD000C3F90321152001F0BFF994F8C83043F080
:102BE000010384F8C830BDE81040FFF709BC10BDF0
:102BF000003802402DE9F04700F5805588B095F87F
:102C0000C930012B0446884616467FD8804F57F8B6
:102C100023200AB947F82300D7F800A0C4F80C8095
:102C20002674BAF1000F63D095F8C930012B6FD02C
:102C300001212046FFF7AAFFFFF7DCFB626913685A
:102C400023F0020313606269136843F00103136009
:102C5000636900275F6101212046FFF7D1FBFFF781
:102C6000F7FD002800F09580E86DFFF793FA04F572
:102C70008359BA4609F10809202200216846FEF767
:102C80005BFF02A8FFF782FCCDF818A06A4609EBAB
:102C900007030DF1180E9446BCE80300F4451860D4
:102CA0005960624603F10803F5D1DCF800001860B2
:102CB00020379CF804201A71602FDDD195F8C830B8
:102CC0006FF38203002785F8C8306A4641462046E4
:102CD000ADF80070ADF802708DF80470FFF75CFD80
:102CE000636948BB4FF400421A6008B0BDE8F08742
:102CF00041F2D00003F0DAFC814610B15146FFF7F3
:102D0000E9FCC7F80090B9F1000F8DD10020ECE785
:102D1000386803681B6B98470146002888D13868DB
:102D2000FFF734FF3868036832465B6841469847CE
:102D300000287FF47DAFE9E761221A609DF8023038
:102D40009DF803201B06120402F4702203F0407366
:102D50001343BDF80020C2F3090213439DF8042079
:102D60001205022E02F4E0020CBF4FF000410021D8
:102D7000134362690B43D361636913225A61626929
:102D8000136823F00103136039462046FFF760FD06
:102D900008B96369A6E795F8C93093BB6169D1F8B2
:102DA000002242F00102C1F800226169D1F800223C
:102DB00022F47C5222F00E02C1F800226169D1F89F
:102DC000002242F46062C1F800226269C2F8143243
:102DD0006269C2F80432626941F6FF71C2F80C12EE
:102DE0006269C2F840326269C2F844326369012202
:102DF000C3F81C226269D2F8003223F00103C2F842
:102E0000003295F8C83043F0020385F8C8306CE70B
:102E1000584B002008B500F051F850EA0103024673
:102E200002D0421E61F10001044B186810B10B463C
:102E3000FFF744FDBDE8084001F064B8584B00209E
:102E400008B50020FFF7E8FDBDE8084001F05AB8DA
:102E500008B50120FFF7E0FDBDE8084001F052B8D9
:102E600000B59BB0EFF3098168226846FEF73EFE8D
:102E7000EFF30583014B9B6BFEE700BF00ED00E025
:102E800008B5FFF7EDFF000000B59BB0EFF3098137
:102E900068226846FEF72AFEEFF30583014B5B6B61
:102EA000FEE700BF00ED00E0FEE700000FB408B54C
:102EB000029801F03DFDFEE702F0D2B902F0AAB996
:102EC00013B56C4684E80600031D94E8030083E80C
:102ED0000500012002B010BD73B58568019155B1A0
:102EE0001B885B0707D4D0E900369B6B9847019A93
:102EF000C1B23046A847012002B070BDF0B5866867
:102F000089B005460C465EB1BDF838305B070AD47F
:102F1000D0E900379B6B98472246C1B23846B0478C
:102F2000012009B0F0BD00220023CDE900230023D9
:102F3000ADF808300A4603AB01F108061068516885
:102F40001C4603C40832B2422346F7D11068206001
:102F50009288A280FFF7B2FF0423ADF808302B68F7
:102F6000CDE90001DB6B694628469847D8E70000A9
:102F700030B503680968DD0FB5EBD17F23F06044FD
:102F800021F060424FEAD1700BD0002BB8BFA40CE7
:102F90000029B8BF920C944202D034BF0120002017
:102FA00030BD944205D1C1F38070C3F38073834276
:102FB000F6D194422CBF00200120F1E72DE9F04129
:102FC000456A15B94162BDE8F0814B6823F060475E
:102FD000C3F38A464FEAD37EC3F3807816EA23060A
:102FE00038BF3E46AC462B465A68BEEBD27F22F035
:102FF00060440AD0002A18DAA40CB44217D19D42CA
:103000000FD10D60DEE71346EEE7A74207D102F0CD
:103010008044C2F3807242450BD054B1EFE708D22E
:10302000EDE7CCF800100B60CDE7B44201D0B4421C
:10303000E5D81A689C46002AE5D11960C3E700006C
:103040002DE9F047089D01F007044FEAD508224416
:1030500005F0070500EBD1004FF47F49944201D100
:10306000BDE8F08704F0070705F0070A57453E461C
:1030700038BF5646C6F10806111B8E4228BF0E46C1
:10308000E10808EBD50E415C13F80EC0B94029FAEF
:1030900006F721FA0AF1FFB28CEA010147FA0AF7B2
:1030A00039408CEA010C03F80EC034443544D5E7AE
:1030B00080EA0120082341F2210201B240000029E8
:1030C00080B203F1FF33B8BF504013F0FF03F4D1D7
:1030D0007047000038B50C468D18A54200D138BDA8
:1030E00014F8011BFFF7E4FFF7E7000042684AB15C
:1030F000136843604389818901339BB299424381BC
:1031000038BF83811046704770B588B020220446CE
:103110000D4668460021FEF70FFD20460495FFF797
:10312000E5FF024658B16B46054608AE1C4603CC87
:10313000B44228606960234605F10805F6D11046BF
:1031400008B070BD082817D909280CD00A280CD05F
:103150000B280CD00C280CD00D280CD00E2814BF36
:103160004020302070470C207047102070471420FA
:10317000704718207047202070470000082817D992
:103180000C280CD910280CD914280CD918280CD9C3
:1031900020280CD930288CBF0F200E207047092022
:1031A00070470A2070470B2070470C2070470D2095
:1031B000704700002DE9F843078C072F04461ED9FD
:1031C000D0E9029800254FF6FF73C5F12006A5F15E
:1031D000200029FA05F108FA06F628FA00F0314332
:1031E0000143C9B21846FFF763FF0835402D034677
:1031F000EBD1E1693A46BDE8F843FFF76BBF4FF604
:10320000FF70BDE8F883000010B54B6823B9CA8A87
:1032100063F30902CA8210BD04691A681C60036165
:10322000C38A013BC3824A60EFE700002DE9F84FF3
:103230001D46CB8A0F46C3F30901052981469246F4
:103240000B4630D00020AAB207F11A049EB2042E19
:103250001FFA80F80FD8904503F1010306D3FB8ACB
:103260000A4462F30903FB8201201AE01AF80060A5
:10327000E6540130EAE79045F1D2A1F1050B1C2399
:103280007C68BBFBF3F203FB12BB1FFA8BF6002C2E
:1032900045D14846FFF72AFF044638B978606FF0F9
:1032A0000200BDE8F88F4FF00008E6E70026066050
:1032B0007860ADB24FF0000B454510D90AEB08031A
:1032C000221D13F8011B9155B1B208F101081B2909
:1032D0001FFA88F82BD0454506F10106F1D8FB8A84
:1032E000C3F30902154465F30903BCE7013292B246
:1032F0001C462368002BF9D16B1F0B441C21B3FB28
:10330000F1F301339BB29A42D3D2BBF1000FD0D17B
:103310004846FFF7EBFE20B9C4F800B0BFE7012232
:10332000E7E7C0F800B05E4620600446C1E74545C7
:10333000D5D94846FFF7DAFE08B92060AFE7C0F8F4
:1033400000B0002620600446B6E700002DE9F04FEB
:103350002DED028B1C4683B05B69019207468846BF
:10336000002B00F09A80238C2BB1E269002A00F038
:103370009480072B35D807F10C00FFF7B7FE054600
:1033800038B96FF00205284603B0BDEC028BBDE8EA
:10339000F08F14220021FEF7CFFB228CE16905F1AA
:1033A0000800FEF7A3FB208C013080B2FFF7E6FE99
:1033B000FFF7C8FE013880B22084013028746369A9
:1033C000228C1B782A4403F01F0363F03F0348F06C
:1033D00000411372384669602946FFF7EFFD012569
:1033E000D1E700F10C034FF0000908EE103A4FF05E
:1033F000800A4E464D4618EE100AFFF777FE8346C8
:103400000028BED014220021FEF796FB002E3AD1F0
:10341000019BABF8083002220BF1080E1FFA82FC68
:103420000CF10100BCF1060F218C80B201D88E4254
:103430002BD3FFF7A3FEFFF785FE626912780138F0
:1034400002F01F028E4208BF4FF0400A42EA4912C2
:103450001BFA80F14AEA020A013048F0004281F882
:1034600008A08BF81000CBF8042059463846FFF727
:10347000A5FD238C0135B3422DB289F001094FF02F
:10348000000AB8D17FE70022C6E7E169895D0EF83E
:1034900002100136B6B20132C0E76FF0010572E7E3
:1034A000F8B515460E463022002104461F46FEF7A9
:1034B00043FB069B6360B5F5001F079BA76034BF05
:1034C0006A094FF6FF72A36297B2E66104F1100039
:1034D00000239A4206D800230360A782E382238355
:1034E000E360F8BD0660013330462036F1E70000A6
:1034F00003781BB94BB2002BC8BF017070470000A6
:1035000000787047F8B50C46C969074611B9238C95
:10351000002B37D1257E1F2D34D8387828BB228C3C
:10352000072A2CD8268A36F003032BD14FF6FF70DA
:10353000FFF7D0FD20F001003102400441EA0561AF
:10354000400C41EA40254FF6FF7223462946384693
:10355000FFF7FCFE002807DD626913780133DBB258
:103560001F2B88BF00231370F8BD218A2D0645EA62
:10357000012505432046FFF71DFE0246E5E76FF0F3
:103580000300F1E76FF00100EEE7000070B58AB0CC
:10359000044616460021282268461D46FEF7CCFA4E
:1035A000BDF83830ADF810300F9B05939DF84030D2
:1035B0008DF81830119B07936946BDF84830ADF877
:1035C00020302046CDE90265FFF79CFF0AB070BDB0
:1035D0002DE9F041D36905460C4616460BB9138C0C
:1035E0005BBB377E1F2F28D895F80080B8F1000FFD
:1035F00026D03046FFF7DEFD3378210241EAC331A1
:1036000041EA0801338A41EA076141EA034102467F
:10361000334641F080012846FFF798FE00280ADD76
:103620003378012B07D1726913780133DBB21F2B7A
:1036300088BF00231370BDE8F0816FF00100FAE746
:103640006FF00300F7E70000F0B58BB004460D46BD
:1036500017460021282268461E46FEF76DFA9DF89F
:103660004C305A1E534253418DF800309DF8403083
:10367000ADF81030119B05939DF848308DF8183047
:10368000149B07936A46BDF85430ADF820302946A4
:103690002046CDE90276FFF79BFF0BB0F0BD00009E
:1036A000406A00B104307047436A1A684262026996
:1036B0001A600361C38A013BC38270472DE9F04160
:1036C000D0F82080194E14461D464146002709B9FE
:1036D000BDE8F081D1E90223A21A65EB030396420B
:1036E00077EB03031ED2036A8B420DD1FFF78CFDEB
:1036F000036A1B68036203690B60C38A0161016A84
:10370000013BC3828846E2E7FFF77EFD0B68C8F8FD
:10371000003003690B60C38A0161013BC382D8F8A2
:103720000010D4E788460968D1E700BF80841E00F6
:103730002DE9F04F8BB00D46DDF8509014469B46B6
:103740008046002800F01981B9F1000F00F01581C2
:10375000531E3F2B00F21181012A03D1BBF1000F50
:1037600040F00B810023CDE90833B8F81430B5EBF5
:10377000C30F4FEAC30703D300200BB0BDE8F08F9F
:103780002B199F42D8F80C303ABF7F1BFFB2274657
:103790001BB9D8F81030002B7AD0272D4ED8C5F1A0
:1037A0002806B7424FF000032CBFF6B23E46009306
:1037B0002946D8F8080008AB3246FFF741FCA7EBD2
:1037C000060A35445FFA8AFAB8F8143003F1005358
:1037D000053BDB000493D8F80C3003932821039BAE
:1037E00013B1BAF1000F2CD1D8F8100040B1BAF1E2
:1037F000000F05D0009608AB5246691AFFF720FC6F
:1038000038B2002FB8D066070AD00AAB03EBD40158
:10381000624211F8083C02F00702134101F8083C2B
:10382000082C3CD9102C40F2B580202C40F2B780F7
:10383000BBF1000F00F09C80082334E0BA4600265C
:10384000C2E7049BE02B28BFE02306930B44AB4266
:10385000059314D95A1B03980096924534BF5246DB
:10386000D2B2691A08AB04300792FFF7E9FB079A56
:103870001644AAEB020A1544F6B25FFA8AFA049BD0
:10388000069A05999B1A0493039B1B680393A6E76A
:103890000093D8F8080008AB3A462946AEE7BBF1DA
:1038A000000F13D00123B4EBC30F6CD0082C12D837
:1038B0009DF82030621E23FA02F2D50706D54FF09C
:1038C000FF3202FA04F423438DF820309DF82030B3
:1038D00089F8003051E7102C12D8BDF82030621E54
:1038E00023FA02F2D10706D54FF0FF3202FA04F4B0
:1038F0002343ADF82030BDF82030A9F800303CE774
:10390000202C0FD80899631E21FA03F3DA0705D596
:103910004FF0FF3202FA04F40C430894089BC9F8F4
:1039200000302AE7402C2BD0DDE90865611EC4F188
:103930002102A4F1210326FA01F105FA02F225FA87
:1039400003F311431943CB0712D50122A4F120033D
:10395000C4F1200102FA03F322FA01F1A24052421B
:1039600043EA010363EB430332432B43CDE90823CE
:10397000DDE90823C9E90023FFE66FF00100FCE65A
:103980006FF00800F9E6082CA0D9102CB3D9202C30
:10399000EED8C3E7BBF1000FADD0022383E7BBF144
:1039A000000FBBD004237EE730B5012A144638BF90
:1039B0000124402C85B028BF40240025012ACDE9F0
:1039C000025518D81B788DF8083063070AD004AB6D
:1039D00003EBD405624215F8083C02F0070293405D
:1039E00005F8083C009103462246002102A8FFF793
:1039F00027FB05B030BD082AE4D9102A03D81B885C
:103A0000ADF80830E1E7202A8DBFD3E900231B6819
:103A10000293CDE90223D8E710B5CB681BB98B60C0
:103A20000B618B8210BD04691A681C600361C38A34
:103A3000013BC382CA60F0E703064CBFC0F3C0304D
:103A40000220704708B50246FFF7F6FF022806D1AC
:103A50005306C2F30F2001D100F0030008BDC2F3EA
:103A60000740FBE72DE9F04F93B0CDE903230A6847
:103A700004461046FFF7E0FF022814BFC2F30626F3
:103A80000026002A0D46824680F2F28112F0C049DB
:103A900040F0EE81097B002900F0EA81022803D082
:103AA0002378B34240F0E781C2F3046306931046E3
:103AB00002F07F030593FFF7C5FF059B29444FEAFA
:103AC000834848EA0A4848EA4668CE78002300223C
:103AD000CDE90823F309834648EA0008029367D03A
:103AE000059B009302466768534608A92046B847DD
:103AF000002800F0C381276A4FB9414604F10C0049
:103B0000FFF702FB074690B96FF0020054E03B69F3
:103B100098450DD03F68002FF9D1414604F10C00C3
:103B2000FFF7F2FA07460028EED0236A3B602762CF
:103B300097F817C006F01F08CCF3840CACEB080014
:103B40001FFA80FE0028B8BF0EF12000A8EB0C037E
:103B50001FFA83FED7E90221B8BF00B2002B0793FA
:103B6000BEBF0EF120031BB2079352EA010338D007
:103B7000039BDFF824E39A1A049B4FF0000C63EBDD
:103B8000010196457CEB01032BD36B7B97F81AE080
:103B9000734519D1029B002B78D0012821DC78686D
:103BA000F8B9DFF8F0C2944570EB010316D337E0A3
:103BB000276A27B96FF00C0013B0BDE8F08F3B699E
:103BC0009845B5D03F68F4E7B24890427CEB0103DA
:103BD00001D30020F0E7029B002BFAD0079B0F2BAC
:103BE00017DCFA7DB30002F0030203F07C031343F9
:103BF000FB7539462046FFF707FB6B7BBB76029BC4
:103C00003BB9FB7DC3F38402013262F38603FB758B
:103C1000D0E76A7BBB7E9A42DBD1029B002B35D07A
:103C2000B309022B32D0039BBB60049BFB601422C0
:103C300000210DA8FDF780FF039B0A93049B0B93C3
:103C40002B1D0C932B7BADF83EB0013BDBB2ADF8E6
:103C50003C30069B8DF84230059B8DF8433094F83C
:103C60002C308DF840A083F001038DF844308DF89E
:103C70004180A3680AA920469847FB7DC3F38403CB
:103C8000013303F01F039B02FB82A2E7FB7DC6F317
:103C90004012B2EBD31F40F0F480C3F384034345DA
:103CA00040F0F280029A2B7BB609002A4DD0F20731
:103CB0005DD4032B40F2EB80039BBB60049BFB6055
:103CC0002B7BAE1D033BDBB23246394604F10C00C0
:103CD000FFF7ACFA00280CDA39462046FFF794FAD1
:103CE000FB7DC3F38403013303F01F039B02FB82BC
:103CF0000AE7DDE90884AB883B834FF6FF73C9F11F
:103D00002000A9F1200228FA09F104FA00F0014389
:103D100024FA02F211431846C9B2FFF7C9F909F1B2
:103D20000809B9F1400F0346E9D1B8822A7B033A6A
:103D3000D2B23146FFF7CEF9FB7DB882DA43C2F347
:103D4000C01262F3C713FB7543E786B92E1D013B12
:103D5000DBB23246394604F10C00FFF767FA00285F
:103D6000BADB2A7BB88A013AD2B23146E2E7F98A55
:103D7000C1F30901013B0429DAB25BD8281D0023F5
:103D800007F11B069A4208D910F801CB06F801C0CA
:103D9000013101330529DBB2F4D103990A91049969
:103DA0000B91934207F11B010C9138BF04337968E2
:103DB0000D9134BF55FA83F300230E93FB8AADF8BF
:103DC0003EB0C3F309031A44069B8DF84230059BAD
:103DD0008DF8433094F82C30ADF83C2083F001038B
:103DE0008DF8443000238DF840A08DF841807B6031
:103DF0002A7BB88A013A291DFFF76CF93B8BB88200
:103E0000834203D1A3680AA92046984720460AA9FD
:103E1000FFF702FEFB7DBA8AC3F38403013303F08C
:103E20001F039B02FB823B8B9A420CBF00206FF06A
:103E30001000C1E67B68002BAFD0052001E01C30EC
:103E400033461E68002EFAD1091A081D2E1D18448B
:103E500001EB090CBCF11B0F5FFA89F39DD89A4264
:103E60009BD916F8013B00F8013B09F10109EFE786
:103E70006FF00900A0E66FF00A009DE66FF00B00FE
:103E80009AE66FF00D0097E66FF00E0094E66FF083
:103E90000F0091E640420F0080841E00EFF309837B
:103EA00005494A6B22F001024A63683383F30988AB
:103EB000002383F31188704700EF00E0302080F387
:103EC000118862B60C4B0D4AD96821F4E0610904EF
:103ED000090C0A43DA60D3F8FC20094942F08072E9
:103EE000C3F8FC200A6842F001020A602022DA7757
:103EF00083F82200704700BF00ED00E00003FA05E0
:103F0000001000E010B5302383F311880E4B5B687E
:103F100013F4006314D0F1EE103AEFF30984683C17
:103F20004FF08073E361094BDB6B236684F30988F0
:103F300000F0BCFC10B1064BA36110BD054BFBE7C4
:103F400083F31188F9E700BF00ED00E000EF00E027
:103F5000430600084606000800F1604303F561438C
:103F60000901C9B283F80013012200F01F039A402F
:103F700043099B0003F1604303F56143C3F88021CB
:103F80001A607047026843681143016003B1184723
:103F90007047000013B5446BD4F894341A68117854
:103FA000042915D1217C022912D119791289012302
:103FB0008B4013420CD101A904F14C0001F0BAFF6F
:103FC000D4F89444019B21790246206800F0D0F98E
:103FD00002B010BD143001F03DBF00004FF0FF33C0
:103FE000143001F037BF00004C3002F00FB8000071
:103FF0004FF0FF334C3002F009B80000143001F0EC
:104000000BBF00004FF0FF31143001F005BF00007E
:104010004C3001F0DBBF00004FF0FF324C3001F0BC
:10402000D5BF00000020704710B5D0F894341A684E
:1040300011780429044617D1017C022914D1597939
:10404000528901238B4013420ED1143001F09EFEA1
:10405000024648B1D4F894444FF4807361792068E3
:10406000BDE8104000F072B910BD0000406BFFF7D2
:10407000DBBF0000704700007FB5124B03600023D8
:104080004360C0E90233012502260F4B0574044644
:104090000290019300F18402294600964FF4807348
:1040A000143001F04FFE094B0294CDE9006304F592
:1040B00023724FF48073294604F14C0001F016FF7F
:1040C00004B070BD386900086D400008953F0008D5
:1040D0000B68302282F311880A7903EB8202906127
:1040E0004A79093243F822008A7912B103EB82033C
:1040F00098610223C0F894140374002080F311889F
:104100007047000038B5037F044613B190F854306F
:10411000ABB9201D01250221FFF734FF04F1140083
:1041200025776FF0010100F09FFC84F8545004F1F2
:104130004C006FF00101BDE8384000F095BC38BD7F
:1041400010B5012104460430FFF71CFF002323773C
:1041500084F8543010BD000038B5044600251430F2
:1041600001F008FE04F14C00257701F0D7FE201D78
:1041700084F854500121FFF705FF2046BDE8384080
:10418000FFF752BF90F8443003F06003202B07D1B3
:1041900090F84520212A4FF0000303D81F2A06D8A3
:1041A00000207047222AFBD1C0E90E3303E0034A06
:1041B00082630722C2630364012070471D2300202D
:1041C00037B5D0F894341A681178042904461AD106
:1041D000017C022917D11979128901238B401342DE
:1041E00011D100F14C05284601F058FF58B101A942
:1041F000284601F09FFED4F89444019B21790246A1
:10420000206800F0B5F803B030BD0000F0B500EB59
:10421000810385B09E6904460D46FEB1302383F3C9
:10422000118804EB8507301D0821FFF7ABFEFB6802
:104230005B691B6806F14C001BB1019001F088FE20
:10424000019803A901F076FE024648B1039B294676
:10425000204600F08DF8002383F3118805B0F0BDEF
:10426000FB685A691268002AF5D01B8A013B13408B
:10427000F1D104F14402EAE7093138B550F82140A0
:10428000DCB1302383F31188D4F894241368527975
:1042900003EB8203DB689B695D6845B1042160180C
:1042A000FFF770FE294604F1140001F079FD204665
:1042B000FFF7BAFE002383F3118838BD7047000072
:1042C00001F0EEB8012303700023C0E90133C3619C
:1042D00083620362C36243620363704738B5044676
:1042E000302383F311880025C0E90355C0E9055543
:1042F000416001F0E5F80223237085F31188284618
:1043000038BD000070B500EB810305465069DA60E6
:104310000E46144618B110220021FDF70DFCA069CD
:1043200018B110220021FDF707FC31462846BDE8F0
:10433000704001F08FB90000826802F001128260C3
:104340000022C0E90422826101F010BAF0B400EB4F
:1043500081044789E4680125A4698D403D43458176
:1043600023600023A2606360F0BC01F02BBA000060
:10437000F0B400EB81040789E468012564698D408D
:104380003D43058123600023A2606360F0BC01F01F
:10439000A5BA000070B50223002504460370C0E9E9
:1043A0000255C0E90455C564856180F8345001F0B8
:1043B000EDF863681B6823B129462046BDE87040CC
:1043C000184770BD0378052B10B504460AD080F855
:1043D00050300523037043681B680BB104219847D4
:1043E0000023A36010BD00000178052906D190F8D4
:1043F0005020436802701B6803B1184770470000E3
:1044000070B590F83430044613B1002380F834308E
:1044100004F14402204601F0CBF963689B68B3B90C
:1044200094F8443013F0600535D00021204601F0A7
:104430006BFC0021204601F05DFC63681B6813B132
:10444000062120469847062384F8343070BD204664
:1044500098470028E4D0B4F84A30E26B9A4288BF0B
:10446000E36394F94430E56B002B4FF0300380F2A6
:104470000381002D00F0F280092284F8342083F3B8
:1044800011880021D4E90E232046FFF771FF002395
:1044900083F31188DAE794F8452003F07F0343EAB9
:1044A000022340F20232934200F0C58021D8B3F5D6
:1044B000807F48D00DD8012B3FD0022B00F0938095
:1044C000002BB2D104F14C02A2630222E263236406
:1044D000C1E7B3F5817F00F09B80B3F5407FA4D1A5
:1044E00094F84630012BA0D1B4F84C3043F00203CD
:1044F00032E0B3F5006F4DD017D8B3F5A06F31D0CF
:10450000A3F5C063012B90D8636894F846205E68D9
:1045100094F84710B4F848302046B047002884D0BB
:104520004368A3630368E3631AE0B3F5106F36D002
:1045300040F6024293427FF478AF5C4BA3630223C0
:10454000E3630023C3E794F84630012B7FF46DAF9B
:10455000B4F84C3023F00203C4E90E55A4F84C30F3
:10456000256478E7B4F84430B3F5A06F0ED194F821
:10457000463084F84E30204601F060F863681B68CE
:1045800013B1012120469847032323700023C4E977
:104590000E339CE704F14F03A3630123C3E72378A1
:1045A000042B10D1302383F311882046FFF7C4FE7B
:1045B00085F311880321636884F84F5021701B68CC
:1045C0000BB12046984794F84630002BDED084F893
:1045D0004F300423237063681B68002BD6D0022160
:1045E00020469847D2E794F848301D0603F00F01A3
:1045F00020460AD501F0CEF8012804D002287FF425
:1046000014AF2B4B9AE72B4B98E701F0B5F8F3E783
:1046100094F84630002B7FF408AF94F8483013F03C
:104620000F01B3D01A06204602D501F081FBADE799
:1046300001F074FBAAE794F84630002B7FF4F5AE46
:1046400094F8483013F00F01A0D01B06204602D585
:1046500001F05AFB9AE701F04DFB97E7142284F82A
:10466000342083F311882B462A4629462046FFF73B
:104670006DFE85F31188E9E65DB1152284F83420DA
:1046800083F311880021D4E90E232046FFF75EFE54
:10469000FDE60B2284F8342083F311882B462A464A
:1046A00029462046FFF764FEE3E700BF686900087B
:1046B000606900086469000838B590F83430044631
:1046C000002B3ED0063BDAB20F2A34D80F2B32D85B
:1046D000DFE803F037313108223231313131313105
:1046E00031313737C56BB0F84A309D4214D2C368B8
:1046F0001B8AB5FBF3F203FB12556DB9302383F32C
:1047000011882B462A462946FFF732FE85F3118889
:104710000A2384F834300EE0142384F83430302334
:1047200083F3118800231A4619462046FFF70EFE30
:10473000002383F3118838BD036C03B1984700232D
:10474000E7E70021204601F0DFFA0021204601F0D2
:10475000D1FA63681B6813B10621204698470623E7
:10476000D7E7000010B590F83430142B044629D058
:1047700017D8062B05D001D81BB110BD093B022B61
:10478000FBD80021204601F0BFFA0021204601F0AD
:10479000B1FA63681B6813B10621204698470623C7
:1047A00019E0152BE9D10B2380F83430302383F343
:1047B000118800231A461946FFF7DAFD002383F318
:1047C0001188DAE7C3689B695B68002BD5D1036C5D
:1047D00003B19847002384F83430CEE700230375F3
:1047E000826803691B6899689142FBD25A6803602A
:1047F0004260106058607047002303758268036947
:104800001B6899689142FBD85A6803604260106047
:104810005860704708B50846302383F311880B7D34
:10482000032B05D0042B0DD02BB983F3118808BDC1
:104830008B6900221A604FF0FF338361FFF7CEFFD0
:104840000023F2E7D1E9003213605A60F3E7000079
:10485000FFF7C4BF054BD9680875186802681A606D
:10486000536001220275D860FBF7D6BE684B00206A
:1048700030B50C4BDD684B1C87B004460FD02B467F
:10488000094A684600F084F92046FFF7E3FF009BE1
:1048900013B1684600F086F9A86907B030BDFFF78C
:1048A000D9FFF9E7684B002015480008044B1A6847
:1048B000DB6890689B68984294BF00200120704795
:1048C000684B0020084B10B51C68D86822681A6035
:1048D000536001222275DC60FFF78EFF01462046FF
:1048E000BDE81040FBF798BE684B0020044B1A68E7
:1048F000DB6892689B689A4201D9FFF7E3BF704773
:10490000684B002038B5074C0749084801230025AB
:104910002370656001F0FAFB0223237085F3118890
:1049200038BD00BFD04D002070690008684B0020E2
:1049300008B572B6044B186500F050FC00F00EFD8F
:10494000024B03221A70FEE7684B0020D04D002076
:1049500000F05EB9EFF3118020B9EFF30583302248
:1049600082F311887047000010B530B9EFF3058469
:10497000C4F3080414B180F3118810BDFFF7B6FF2B
:1049800084F31188F9E70000034A516853685B1A01
:104990009842FBD8704700BF001000E08B600223F4
:1049A00008618B82084670478368A3F1840243F84C
:1049B000142C026943F8442C426943F8402C094AFC
:1049C00043F8242CC26843F8182C022203F80C2C5C
:1049D000002203F80B2C044A43F8102CA3F120000A
:1049E000704700BF31060008684B002008B5FFF78C
:1049F000DBFFBDE80840FFF72BBF0000024BDB6880
:104A000098610F20FFF726BF684B0020302383F307
:104A10001188FFF7F3BF000008B50146302383F388
:104A200011880820FFF724FF002383F3118808BDB5
:104A3000064BDB6839B1426818605A601360436006
:104A40000420FFF715BF4FF0FF307047684B002080
:104A50000368984206D01A6802605060996118464F
:104A6000FFF7F6BE7047000038B504460D462068D3
:104A7000844200D138BD036823605C608561FFF724
:104A8000E7FEF4E710B503689C68A2420CD85C68A6
:104A90008A600B604C602160596099688A1A9A603C
:104AA0004FF0FF33836010BD1B68121BECE7000062
:104AB0000A2938BF0A2170B504460D460A26601936
:104AC00001F01EFB01F00AFB041BA54203D8751C74
:104AD0002E460446F3E70A2E04D9BDE870400120B3
:104AE00001F054BB70BD0000F8B5144B0D46D96100
:104AF00003F1100141600A2A1969826038BF0A2255
:104B0000016048601861A818144601F0EBFA0A2702
:104B100001F0E4FA431BA342064606D37C1C281985
:104B200001F0EEFA27463546F2E70A2F04D9BDE830
:104B3000F840012001F02ABBF8BD00BF684B0020FF
:104B4000F8B506460D4601F0C9FA0F4A134653F868
:104B5000107F9F4206D12A4601463046BDE8F84004
:104B6000FFF7C2BFD169BB68441A2C1928BF2C4675
:104B7000A34202D92946FFF79BFF2246314603484C
:104B8000BDE8F840FFF77EBF684B0020784B00205F
:104B900010B4C0E9032300235DF8044B4361FFF721
:104BA000CFBF000010B5194C236998420DD0D0E951
:104BB0000032816813605A609A680A449A60002340
:104BC00003604FF0FF33A36110BD2346026843F832
:104BD000102F53600022026022699A4203D1BDE87F
:104BE000104001F087BA936881680B44936001F02C
:104BF00075FA2269E1699268441AA242E4D9114423
:104C0000BDE81040091AFFF753BF00BF684B0020F2
:104C10002DE9F047DFF8BC8008F110072C4ED8F8DA
:104C2000105001F05BFAD8F81C40AA68031B9A42A6
:104C30003ED81444D5E900324FF00009C8F81C40B2
:104C400013605A60C5F80090D8F81030B34201D113
:104C500001F050FA89F31188D5E9033128469847C5
:104C6000302383F311886B69002BD8D001F036FA1A
:104C70006A69A0EB04094A4582460DD2022001F080
:104C800085FA0022D8F81030B34208D151462846A0
:104C9000BDE8F047FFF728BF121A2244F2E712EBF3
:104CA000090938BF4A4629463846FFF7EBFEB5E703
:104CB000D8F81030B34208D01444211AC8F81C00A8
:104CC000A960BDE8F047FFF7F3BEBDE8F08700BF7D
:104CD000784B0020684B002000207047FEE7000062
:104CE000704700004FF0FF307047000002290CD0E1
:104CF000032904D00129074818BF00207047032A60
:104D000005D8054800EBC2007047044870470020F2
:104D1000704700BF486A00082C230020FC69000887
:104D200070B59AB00546084601A9144600F0C2F8CD
:104D300001A8FCF7F9FE431C5B00C5E90034002222
:104D4000237003236370C6B201AB02341046D1B2A4
:104D50008E4204F1020401D81AB070BD13F8011B91
:104D600004F8021C04F8010C0132F0E708B5302306
:104D700083F311880348FFF723FA002383F3118894
:104D800008BD00BFD84D002090F8443003F01F024A
:104D9000012A07D190F845200B2A03D10023C0E94E
:104DA0000E3315E003F06003202B08D1B0F8483033
:104DB0002BB990F84520212A03D81F2A04D8FFF7E1
:104DC000E1B9222AEBD0FAE7034A82630722C263E1
:104DD00003640120704700BF2423002007B5052984
:104DE00017D8DFE801F0191603191920302383F3CF
:104DF0001188104A01900121FFF784FA01980E4AA8
:104E00000221FFF77FFA0D48FFF7A6F9002383F38D
:104E1000118803B05DF804FB302383F31188074841
:104E2000FFF770F9F2E7302383F311880348FFF7A7
:104E300087F9EBE79C690008C0690008D84D00209D
:104E400038B50C4D0C4C0D492A4604F10800FFF70B
:104E500067FF05F1CA0204F110000949FFF760FF7E
:104E600005F5CA7204F118000649BDE83840FFF79D
:104E700057BF00BFA05200202C2300207C690008EF
:104E8000866900089169000870B5044608460D4619
:104E9000FCF74AFEC6B22046013403780BB9184627
:104EA00070BD32462946FCF72BFE0028F3D10120C5
:104EB000F6E700002DE9F04705460C46FCF734FE06
:104EC0002B49C6B22846FFF7DFFF08B10B36F6B212
:104ED00028492846FFF7D8FF08B11036F6B2632EEE
:104EE0000BD8DFF88C80DFF88C90234FDFF894A08C
:104EF0002E7846B92670BDE8F08729462046BDE8E1
:104F0000F04701F091BC252E2ED1072241462846BC
:104F1000FCF7F6FD70B9194B224603F1100153F866
:104F2000040B42F8040B8B42F9D11B881380073520
:104F30001234DDE7082249462846FCF7E1FD98B91E
:104F40000F4BA21C197809090232C95D02F8041C32
:104F500013F8011B01F00F015345C95D02F8031C52
:104F6000F0D118340835C3E704F8016B0135BFE709
:104F7000686A000891690008706A000846680008BD
:104F8000107AFF1F1C7AFF1FBFF34F8F024AD368AE
:104F9000DB03FCD4704700BF003C024008B5094B5E
:104FA0001B7873B9FFF7F0FF074B1A69002ABFBFE0
:104FB000064A5A6002F188325A601A6822F4806206
:104FC0001A6008BDFE540020003C024023016745E2
:104FD00008B50B4B1B7893B9FFF7D6FF094B1A693D
:104FE00042F000421A611A6842F480521A601A684C
:104FF00022F480521A601A6842F480621A6008BD76
:10500000FE540020003C02400B28F0B516D80C4C92
:105010000C4923787BB90C4D0E460C234FF00062EF
:1050200055F8047B46F8042B013B13F0FF033A4488
:10503000F6D10123237051F82000F0BD0020FCE7D9
:105040003055002000550020846A0008014B53F8B9
:1050500020007047846A00080C2070470B2810B5A8
:10506000044601D9002010BDFFF7CEFF064B53F8D0
:1050700024301844C21A0BB90120F4E71268013237
:10508000F0D1043BF6E700BF846A00080B2810B596
:10509000044621D8FFF778FFFFF780FF0F4AF3237C
:1050A000D360C300DBB243F4007343F00203136127
:1050B000136943F480331361FFF766FFFFF7A4FF22
:1050C000074B53F8241000F045F9FFF781FF204605
:1050D000BDE81040FFF7C2BF002010BD003C0240F9
:1050E000846A0008F8B512F00103144642D1821810
:1050F000B2F1016F57D82D4B1B6813F0010352D04A
:105100002B4DFFF74BFFF323EB60FFF73DFF40F222
:105110000127032C15D824F001046618244C401AEA
:1051200040F20117B142236900EB010524D123F0BD
:1051300001032361FFF74CFF0120F8BD043C04305C
:10514000E7E78307E7D12B6923F440732B612B69D1
:105150003B432B6151F8046B0660BFF34F8FFFF7A1
:1051600013FF03689E42E9D02B6923F001032B61F2
:10517000FFF72EFF0020E0E723F44073236123694B
:105180003B4323610B882B80BFF34F8FFFF7FCFE5F
:105190002D8831F8023BADB2AB42C3D0236923F076
:1051A00001032361E4E71846C7E700BF0038024067
:1051B000003C0240084908B50B7828B11BB9FFF73D
:1051C000EDFE01230B7008BD002BFCD0BDE80840AC
:1051D0000870FFF7FDBE00BFFE54002008B54FF475
:1051E00000314FF0005000F0B7F8BDE808404FF430
:1051F00080314FF0805000F0AFB8000008461146F3
:1052000001F076BA012001F073BA0000084601F0FF
:105210008DBA000070B582B0FFF79CFB0E4E0546BC
:1052200000F05CFF3268904237BF0C4A0B4951686E
:1052300014682EBFD1E900410131516004190346C1
:1052400041F10001284601913360FFF78DFB019980
:10525000204602B070BD00BF3455002038550020F4
:1052600070B582B0FFF776FB104E054600F036FFB2
:105270003268904237BF0E4A0D49516814682EBFFC
:10528000D1E9004101315160041941F100010346A7
:10529000284601913360FFF767FB01994FF47A725A
:1052A00000232046FAF7A4FF02B070BD3455002059
:1052B0003855002010B50244064BD2B2904200D1BE
:1052C00010BD441C00B253F8200041F8040BE0B2BA
:1052D000F4E700BF502800400F4B30B51C6F24048A
:1052E00007D41C6F44F400741C671C6F44F4004422
:1052F0001C670A4C236843F4807323600244084B04
:10530000D2B2904200D130BD441C00B251F8045BCF
:1053100043F82050E0B2F4E700380240007000404B
:105320005028004007B5012201A90020FFF7C2FF65
:10533000019803B05DF804FB13B50446FFF7F2FFD4
:10534000A04205D0012201A900200194FFF7C4FF6B
:1053500002B010BD704700007047000070470000A9
:10536000074B45F255521A6002225A6040F6FF720E
:105370009A604CF6CC421A60024B01221A707047B8
:105380000030004044550020034B1B781BB1034BF9
:105390004AF6AA221A6070474455002000300040A7
:1053A000034B1A681AB9034AD2F874281A60704776
:1053B0004055002000300240024B4FF08072C3F88D
:1053C000742870470030024008B5FFF7E9FF024B30
:1053D0001868C0F3407008BD4055002008B5FFF7BD
:1053E000DFFF024B1868C0F3007008BD4055002075
:1053F00070470000FEE700000A4B0B480B4A904242
:105400000BD30B4BDA1C121AC11E22F003028B4283
:1054100038BF00220021FCF78FBB53F8041B40F873
:10542000041BECE7A86C00084856002048560020F2
:105430004856002070B5D0E915439E6800224FF011
:10544000FF3504EB42135101D3F800090028BEBF19
:10545000D3F8000940F08040C3F80009D3F8000BEE
:105460000028BEBFD3F8000B40F08040C3F8000B0B
:10547000013263189642C3F80859C3F8085BE0D2BA
:105480004FF00113C4F81C3870BD0000890141F0D1
:105490002001016103699B06FCD41220FFF774BA56
:1054A00010B5054C2046FEF70DFF4FF0A043636595
:1054B000024BA36510BD00BF48550020D86A000804
:1054C00070B50378012B054650D12A4B446D9842A4
:1054D0001BD1294B5A6B42F080025A635A6D42F03D
:1054E00080025A655A6D5A6942F080025A615A69BF
:1054F00022F080025A610E2143205B69FEF72CFDE9
:105500001E4BE3601E4BC4F800380023C4F8003E75
:10551000C02323606E6D4FF40413A3633369002B23
:10552000FCDA012333610C20FFF72EFA3369DB0725
:10553000FCD41220FFF728FA3369002BFCDA00268E
:10554000A6602846FFF776FF6B68C4F81068DB6832
:10555000C4F81468C4F81C684BB90A4BA3614FF037
:10556000FF336361A36843F00103A36070BD064B82
:10557000F4E700BF485500200038024040140040C6
:1055800003002002003C30C0083C30C0F8B5446D38
:10559000054600212046FFF779FFA96D00234FF053
:1055A00001128F68C4F834384FF00066C4F81C2824
:1055B0004FF0FF3004EB431201339F42C2F8006901
:1055C000C2F8006BC2F80809C2F8080BF2D20B68E7
:1055D0006A6DEB65636210231361166916F010069D
:1055E000FBD11220FFF7D0F9D4F8003823F4FE6382
:1055F000C4F80038A36943F4402343F01003A361C7
:105600000923C4F81038C4F814380A4BEB604FF083
:10561000C043C4F8103B084BC4F8003BC4F8106901
:10562000C4F80039EB6D03F1100243F48013EA650E
:10563000A362F8BDB46A000840800010426D90F883
:105640004E10D2F8003823F4FE6343EA0113C2F887
:10565000003870472DE9F84300EB8103456DDA68A7
:10566000166806F00306731E022B05EB41130C4669
:1056700080460FFA81F94FEA41104FF00001C3F85C
:10568000101B4FF0010104F1100398BFB60401FA9A
:1056900003F391698EBF334E06F1805606F500463E
:1056A00000293AD0578A04F15801490137436F5015
:1056B000D5F81C180B43C5F81C382B180021C3F86B
:1056C000101953690127611EA7409BB3138A928B5F
:1056D0009B08012A88BF5343D8F85C20981842EAF7
:1056E000034301F1400205EB8202C8F85C00214649
:1056F00053602846FFF7CAFE08EB8900C3681B8A7F
:1057000043EA8453483464011E432E51D5F81C38B3
:105710001F43C5F81C78BDE8F88305EB4917D7F897
:10572000001B21F40041C7F8001BD5F81C1821EA22
:105730000303C0E704F13F0305EB83030A4A5A6001
:1057400028462146FFF7A2FE05EB4910D0F80039A4
:1057500023F40043C0F80039D5F81C3823EA0707C2
:10576000D7E700BF0080001000040002826D1268BD
:10577000C265FFF75FBE00005831436D49015B58B9
:1057800013F4004004D013F4001F0CBF02200120CA
:10579000704700004831436D49015B5813F40040E5
:1057A00004D013F4001F0CBF02200120704700003A
:1057B00000EB8101CB68196A0B6813604B6853607A
:1057C0007047000000EB810330B5DD68AA691368FB
:1057D000D36019B9402B84BF402313606B8A1468CF
:1057E000426D1C44013CB4FBF3F46343033323F0E8
:1057F000030302EB411043EAC44343F0C043C0F843
:10580000103B2B6803F00303012B09B20ED1D2F831
:10581000083802EB411013F4807FD0F8003B14BF2E
:1058200043F0805343F00053C0F8003B02EB4112B9
:10583000D2F8003B43F00443C2F8003B30BD000007
:105840002DE9F041244D6E6D06EB40130446D3F86C
:10585000087BC3F8087B38070AD5D6F8143819072F
:1058600006D505EB84032146DB6828465B6898472C
:10587000FA071FD5D6F81438DB071BD505EB8403D0
:10588000D968CCB98B69488A5A68B2FBF0F600FB3C
:1058900016228AB91868DA6890420DD2121AC3E942
:1058A0000024302383F311880B482146FFF78AFF39
:1058B00084F31188BDE8F081012303FA04F26B89B7
:1058C00023EA02036B81CB68002BF3D02146024808
:1058D000BDE8F041184700BF4855002000EB8103A8
:1058E00070B5DD68436D6C692668E6604A0156BB99
:1058F0001A444FF40020C2F810092A6802F003028B
:10590000012A0AB20ED1D3F8080803EB421410F4AE
:10591000807FD4F8000914BF40F0805040F0005060
:10592000C4F8000903EB4212D2F8000940F0044029
:10593000C2F80009D3F83408012202FA01F1014348
:10594000C3F8341870BD19B9402E84BF40202060C0
:1059500020682E8A8419013CB4FBF6F440EAC44066
:1059600040F000501A44C6E72DE9F8433B4D6E6DF8
:1059700006EB40130446D3F80889C3F8088918F0E9
:10598000010F4FEA40171AD0D6F81038DB0716D5AA
:1059900005EB8003D9684B691868DA68904230D209
:1059A000121A4FF000091A60C3F80490302383F3F1
:1059B000118821462846FFF791FF89F3118818F0D6
:1059C000800F1CD0D6F834380126A640334216D0BA
:1059D00005EB84036D6DD3F80CC0DCF814200134A2
:1059E000E4B2D2F800E005EB04342F44516871456D
:1059F00015D3D5F8343823EA0606C5F83468BDE86F
:105A0000F883012303FA04F22B8923EA02032B8192
:105A10008B68002BD3D0214628469847CFE7BCF8A7
:105A20001000AEEB0103834228BF0346D7F81809E4
:105A300080B2B3EB800FE2D89068A0F1040959F866
:105A4000048FC4F80080A0EB09089844B8F1040F53
:105A5000F5D818440B4490605360C7E748550020C0
:105A60002DE9F74FA24C656D6E69AB691E4016F4C7
:105A700080586E6107D02046FEF78CFC03B0BDE86D
:105A8000F04FFEF73FBA002E12DAD5F8003E9848E4
:105A90009B071EBFD5F8003E23F00303C5F8003E68
:105AA000D5F8043823F00103C5F80438FEF79CFC50
:105AB000370505D58E48FFF7BDFC8D48FEF782FC03
:105AC000B0040CD5D5F8083813F0060FEB6823F4B2
:105AD00070530CBF43F4105343F4A053EB603107F1
:105AE0001BD56368DB681BB9AB6923F00803AB61A6
:105AF0002378052B0CD1D5F8003E7D489A071EBFB0
:105B0000D5F8003E23F00303C5F8003EFEF76CFC19
:105B10006368DB680BB176489847F30274D4B70228
:105B200027D5D4F85490DFF8C8B100274FF0010A08
:105B300009EB4712D2F8003B03F44023B3F5802F62
:105B400011D1D2F8003B002B0DDA62890AFA07F373
:105B500022EA0303638104EB8703DB68DB6813B18C
:105B6000394658469847A36D01379B68FFB29F425C
:105B7000DED9F00617D5676D3A6AC2F30A1002F053
:105B80000F0302F4F012B2F5802F00F08580B2F519
:105B9000402F08D104EB83030022DB681B6A07F562
:105BA000805790426AD13003D5F8184813D5E103E5
:105BB00002D50020FFF744FEA20302D50120FFF723
:105BC0003FFE630302D50220FFF73AFE270302D50A
:105BD0000320FFF735FE75037FF550AFE00702D5D0
:105BE0000020FFF7C1FEA10702D50120FFF7BCFE90
:105BF000620702D50220FFF7B7FE23077FF53EAF0D
:105C00000320FFF7B1FE39E7636DDFF8E4A00193ED
:105C100000274FF00109A36D9B685FFA87FB9B4546
:105C20003FF67DAF019B03EB4B13D3F8001901F452
:105C30004021B1F5802F1FD1D3F8001900291BDABC
:105C4000D3F8001941F09041C3F80019D3F80019B6
:105C50000029FBDB5946606DFFF718FC218909FA22
:105C60000BF321EA0303238104EB8B03DB689B68BE
:105C700013B15946504698470137CCE7910708BF02
:105C8000D7F80080072A98BF03F8018B02F10102C0
:105C900098BF4FEA182884E7023304EB830207F524
:105CA00080575268D2F818C0DCF80820DCE9001CE4
:105CB000A1EB0C0C002188420AD104EB8304636839
:105CC0009B699A6802449A605A6802445A606AE77B
:105CD00011F0030F08BFD7F800808C4588BF02F889
:105CE000018B01F1010188BF4FEA1828E3E700BFEB
:105CF00048550020436D03EB4111D1F8003B43F4BC
:105D00000013C1F8003B7047436D03EB4111D1F81C
:105D1000003943F40013C1F800397047436D03EBB9
:105D20004111D1F8003B23F40013C1F8003B704748
:105D3000436D03EB4111D1F8003923F40013C1F88E
:105D40000039704730B5039C0172043304FB03250E
:105D5000C0E90653049B03630021059BC160C0E9B1
:105D60000000C0E90422C0E90842C0E90A11436307
:105D700030BD0000416A0022C0E90411C0E90A22D6
:105D8000C2606FF00101FEF76FBE0000D0E904327F
:105D9000934201D1C2680AB9181D704700207047AC
:105DA00003691960C2680132C260C2691344826922
:105DB0000361934224BF436A03610021FEF748BE9A
:105DC00038B504460D46E3683BB16269131D12689D
:105DD000A3621344E362002007E0237A33B9294623
:105DE0002046FEF725FE0028EDDA38BD6FF00100F1
:105DF000FBE70000C368C269013BC3604369134409
:105E000082694361934224BF436A436100238362F2
:105E1000036B03B11847704770B53023044683F312
:105E20001188866A3EB9FFF7CBFF054618B186F3A5
:105E30001188284670BDA36AE26A13F8015BA36269
:105E4000934202D32046FFF7D5FF002383F3118846
:105E5000EFE700002DE9F84F04460E461746984636
:105E60004FF0300989F311880025AA46D4F828B0EC
:105E7000BBF1000F09D141462046FFF7A1FF20B139
:105E80008BF311882846BDE8F88FD4E90A12A7EBF6
:105E9000050B521A934528BF9346BBF1400F1BD9FF
:105EA000334601F1400251F8040B43F8040B9142D0
:105EB000F9D1A36A40334036A3624035D4E90A23BE
:105EC0009A4202D32046FFF795FF8AF31188BD421C
:105ED000D8D289F31188C9E730465A46FBF706FE47
:105EE000A36A5B445E44A3625D44E7E710B5029C8D
:105EF0000172043303FB0421C0E906130023C0E947
:105F00000A33039B0363049BC460C0E90000C0E93B
:105F10000422C0E90842436310BD0000026AC26067
:105F2000426AC0E904220022C0E90A226FF001019E
:105F3000FEF79ABDD0E904239A4201D1C26822B982
:105F4000184650F8043B0B60704700231846FAE7E8
:105F5000C368C2690133C360436913448269436102
:105F6000934224BF436A43610021FEF771BD0000E4
:105F700038B504460D46E3683BB123691A1DA26299
:105F8000E2691344E362002007E0237A33B929462B
:105F90002046FEF74DFD0028EDDA38BD6FF0010018
:105FA000FBE7000003691960C268013AC260C26978
:105FB000134482690361934224BF436A036100234F
:105FC0008362036B03B118477047000070B530233C
:105FD0000D460446114683F31188866A2EB9FFF7F1
:105FE000C7FF10B186F3118870BDA36A1D70A36A44
:105FF000E26A01339342A36204D3E1692046043983
:10600000FFF7D0FF002080F31188EDE72DE9F84F6E
:1060100004460D46904699464FF0300A8AF311889F
:106020000026B346A76A4FB949462046FFF7A0FFAE
:1060300020B187F311883046BDE8F88FD4E90A070C
:106040003A1AA8EB0607974228BF1746402F1BD9DC
:1060500005F1400355F8042B40F8042B9D42F9D17B
:10606000A36A4033A3624036D4E90A239A4204D398
:10607000E16920460439FFF795FF8BF31188464507
:10608000D9D28AF31188CDE729463A46FBF72EFD8F
:10609000A36A3B443D44A3623E44E5E7D0E90423C0
:1060A0009A4217D1C3689BB1836A8BB1043B9B1A98
:1060B0000ED01360C368013BC360C3691A4483698F
:1060C00002619A4224BF436A036100238362012371
:1060D000184670470023FBE700F0D2B84FF080432A
:1060E000586A70474FF08043002258631A610222B9
:1060F000DA6070474FF080430022DA60704700009A
:106100004FF0804358637047FEE7000070B51B4BAB
:1061100001630025044686B0586085620E46FDF78F
:10612000CDFE04F11003C4E904334FF0FF33C4E99A
:106130000635C4E90044A560E562FFF7CFFF2B46B2
:106140000246C4E9082304F134010D4A2565802381
:106150002046FEF723FC0123E0600A4A0375009203
:1061600072680192B268CDE90223074B6846CDE917
:106170000435FEF73BFC06B070BD00BFD04D0020DB
:10618000E46A0008E96A000809610008024AD36A63
:106190001843D062704700BF684B00204B684360D3
:1061A0008B688360CB68C3600B6943614B69036292
:1061B0008B6943620B6803607047000008B5264B8B
:1061C00026481A6940F2FF110A431A611A6922F43B
:1061D000FF7222F001021A611A691A6B0A431A63EC
:1061E0001A6D0A431A651E4A1B6D1146FFF7D6FF4A
:1061F00002F11C0100F58060FFF7D0FF02F13801C9
:1062000000F58060FFF7CAFF02F1540100F58060DD
:10621000FFF7C4FF02F1700100F58060FFF7BEFFD9
:1062200002F18C0100F58060FFF7B8FF02F1A801D0
:1062300000F58060FFF7B2FF02F1C40100F5806055
:10624000FFF7ACFF02F1E00100F58060FFF7A6FF69
:10625000BDE8084000F090B800380240000002405D
:10626000F06A000808B500F0FBF9FEF74BFBFFF7FA
:1062700097F8BDE80840FEF7E3BD00007047000056
:106280000F4B1A6C42F001021A641A6E42F00102BE
:106290001A660C4A1B6E936843F0010393604FF03B
:1062A000804353229A624FF0FF32DA6200229A61F1
:1062B0005A63DA605A6001225A611A60704700BF5F
:1062C00000380240002004E04FF0804208B5116918
:1062D000D3680B40D9B2C9439B07116107D530235E
:1062E00083F31188FEF734FB002383F3118808BD84
:1062F0001F4B1A696FEAC2526FEAD2521A611A69C9
:10630000C2F308021A614FF0FF301A695A695861E6
:1063100000215A6959615A691A6A62F080521A62F8
:106320001A6A02F080521A621A6A5A6A58625A6AE3
:1063300059625A6A1A6C42F080521A641A6E42F01C
:1063400080521A661A6E0B4A106840F48070106012
:10635000186F00F44070B0F5007F1EBF4FF480301E
:1063600018671967536823F40073536000F054B939
:106370000038024000700040334B4FF080521A64E6
:10638000324A4FF4404111601A6842F001021A602B
:106390001A689107FCD59A6822F003029A602A4B8A
:1063A0009A6812F00C02FBD1196801F0F90119602A
:1063B0009A601A6842F480321A601A689203FCD517
:1063C0005A6F42F001025A671F4B5A6F9007FCD573
:1063D0001F4A5A601A6842F080721A601B4A53685A
:1063E0005904FCD5184B1A689201FCD5194A9A60D9
:1063F000194B1A68194B9A42194B21D1194A116845
:10640000194A91421CD140F205121A60144A1368CD
:1064100003F00F03052BFAD10B4B9A6842F00202EE
:106420009A609A6802F00C02082AFAD15A6C42F477
:1064300080425A645A6E42F480425A665B6E7047DC
:1064400040F20572E1E700BF0038024000700040F2
:106450000854400700948838002004E011640020AC
:10646000003C024000ED00E041C20F41074A08B580
:10647000536903F00103536123B1054A13680BB15B
:1064800050689847BDE80840FDF73CBD003C01401E
:10649000C0550020074A08B5536903F00203536151
:1064A00023B1054A93680BB1D0689847BDE808400E
:1064B000FDF728BD003C0140C0550020074A08B543
:1064C000536903F00403536123B1054A13690BB107
:1064D00050699847BDE80840FDF714BD003C0140F5
:1064E000C0550020074A08B5536903F008035361FB
:1064F00023B1054A93690BB1D0699847BDE80840BC
:10650000FDF700BD003C0140C0550020074A08B51A
:10651000536903F01003536123B1054A136A0BB1A9
:10652000506A9847BDE80840FDF7ECBC003C0140CC
:10653000C0550020164B10B55C6904F478725A619E
:10654000A30604D5134A936A0BB1D06A9847600634
:1065500004D5104A136B0BB1506B9847210604D534
:106560000C4A936B0BB1D06B9847E20504D5094AEE
:10657000136C0BB1506C9847A30504D5054A936C76
:106580000BB1D06C9847BDE81040FDF7BBBC00BF15
:10659000003C0140C0550020194B10B55C6904F463
:1065A0007C425A61620504D5164A136D0BB1506DD9
:1065B0009847230504D5134A936D0BB1D06D9847C6
:1065C000E00404D50F4A136E0BB1506E9847A10436
:1065D00004D50C4A936E0BB1D06E9847620404D573
:1065E000084A136F0BB1506F9847230404D5054A2E
:1065F000936F0BB1D06F9847BDE81040FDF782BC98
:10660000003C0140C055002008B5FFF75DFEBDE825
:106610000840FDF777BC0000062108B50846FDF7E5
:106620009BFC06210720FDF797FC06210820FDF7BB
:1066300093FC06210920FDF78FFC06210A20FDF7B7
:106640008BFC06211720FDF787FC06212820FDF78B
:1066500083FCBDE8084007211C20FDF77DBC00003D
:1066600008B5FFF745FE00F00BF8FDF729FEFDF732
:1066700001FDFFF703FEBDE80840FFF72DBD000058
:106680000023054A19460133102BC2E9001102F11B
:106690000802F8D1704700BFC05500200B460146E4
:1066A000184600F02DB8000000F040B8012838BFAF
:1066B000012010B50446204600F030F830B900F053
:1066C00007F808B900F00CF88047F4E710BD0000A7
:1066D000024B1868BFF35B8F704700BF4056002025
:1066E00008B5062000F084F80120FEF7F7FA000054
:1066F000024B0A4601461868FEF780BD4C23002075
:1067000010B5054C13462CB10A4601460220AFF3E2
:10671000008010BD2046FCE700000000024B01464F
:106720001868FEF76FBD00BF4C230020024B0146E6
:106730001868FEF76BBD00BF4C23002010B501396F
:106740000244904201D1002005E0037811F8014F86
:10675000A34201D0181B10BD0130F2E72DE9F04132
:10676000A3B1C91A17780144044603F1FF3C8C42D7
:10677000204601D9002009E00578BD4204F101045A
:10678000F5D10CEB0405D618A54201D1BDE8F08186
:1067900015F8018D16F801EDF045F5D0E7E700009A
:1067A0001F2938B504460D4604D9162303604FF05F
:1067B000FF3038BD426C12B152F821304BB920463F
:1067C00000F030F82A4601462046BDE8384000F087
:1067D00017B8012B0AD0591C03D1162303600120DE
:1067E000E7E7002442F82540284698470020E0E7E4
:1067F000024B01461868FFF7D3BF00BF4C230020AF
:1068000038B5074D00230446084611462B60FEF7B5
:1068100069FA431C02D12B6803B1236038BD00BF65
:1068200044560020FEF758BA034611F8012B03F82E
:10683000012B002AF9D170476F72672E617264755F
:1068400070696C6F742E663430352D4D6174656BD4
:1068500041697273706565640000000053544D33E4
:1068600032463F3F3F0053544D3332463430780078
:1068700053544D3332463432780053544D333246FC
:106880003434365858000000012033000010410015
:1068900001105A00031059000710310000000000D9
:1068A0005C68000813040000666800081904000012
:1068B00070680008210400007A68000840A2E4F132
:1068C000646891060041A3E5F26569920700000043
:1068D0004261642043414E496661636520696E648C
:1068E00065782E008000000000800000000080001D
:1068F00000000000000000000D240008F52B000837
:10690000552B00081D240008512400084D260008BE
:106910002124000831240008252400082D24000823
:10692000292400087525000835240008C12E000818
:10693000452400084925000800000000F13F000838
:10694000DD3F00081940000805400008114000081C
:10695000FD3F0008E93F0008D53F0008254000083A
:106960000000000001000000000000006330000093
:106970006C690008C04B0020D04D00204172647546
:1069800050696C6F740025424F415244252D424C92
:10699000002553455249414C2500000002000000EB
:1069A000000000000D42000879420008400040004D
:1069B0007052002080520020020000000000000001
:1069C0000300000000000000BD42000800000000BD
:1069D00010000000905200200000000001000000A4
:1069E000000000004855002001010200DD4D0008B4
:1069F000ED4C0008894D00086D4D00084300000073
:106A0000046A000809024300020100C032090400C0
:106A1000000102020100052400100105240100010B
:106A2000042402020524060001070582030800FF72
:106A300009040100020A00000007050102400000ED
:106A4000070581024000000012000000506A0008A3
:106A50001201100102000040091241570002010218
:106A6000030100000403090425424F41524425005C
:106A70003031323334353637383941424344454674
:106A80000000000000400000004000000040000046
:106A900000400000000001000000020000000200B1
:106AA00000000200000002000000020000000200DE
:106AB000000002000000000001440008B946000880
:106AC0006547000840004000A8550020A855002058
:106AD00001000000B85500208000000040010000C7
:106AE000030000006D61696E0069646C6500000060
:106AF000AA01A81200000000AAAAAAAA550114001F
:106B0000FFBF00008877000070A70A0000000A019C
:106B100000000000AAAAAAAA00000001FFFF0000CE
:106B200000000000990000000000A0160000000016
:106B3000AAAAAAA600005011FFDF00000000000072
:106B4000007708002000000000000000AAAAAAAAFE
:106B500010000000FFFF000000080000000000001F
:106B60000000000000000000AAAAAAAA000000007D
:106B7000FFFF000000000000000000000000000017
:106B800000000000AAAAAAAA00000000FFFF00005F
:106B900000000000000000000000000000000000F5
:106BA000AAAAAAAA00000000FFFF0000000000003F
:106BB0000000000000000000000000000A000000CB
:106BC00000000000030000000000000000000000C2
:106BD00000000000000000000000000000000000B5
:106BE0000000000000000000000000003496FF7F5D
:106BF0000100000000000000F6030000000000009B
:106C000000000F000000000040420F00FE2A0100BB
:106C1000D2040000FF00960000000008009600006B
:106C20000000080004000000646A00080000000082
:106C30000000000000000000000000000000000054
:106C400000000000502300200000000000000000B1
:106C50000000000000000000000000000000000034
:106C60000000000000000000000000000000000024
:106C70000000000000000000000000000000000014
:106C80000000000000000000000000000000000004
:106C900000000000000000000000000000000000F4
:086CA0000000000000000000EC
:00000001FF
